:020000040800F2
:10500000F81B0020D5500008D18B0008E182000871
:105010000000000000000000000000000000000090
:105020000000000000000000000000002D9A0008B1
:105030000000000000000000A9930008699B000820
:10504000E7500008E7500008E7500008E750000864
:10505000E7500008D95C0008E7500008E750000856
:1050600000000000E7500008015C0008E75000085D
:10507000E7500008C187000800000000E750000862
:1050800000000000E75000080000000000000000E1
:10509000E750000800000000E7500008E750000853
:1050A000E7500008E7500008E7500008E5A50008B1
:1050B000E7500008E7500008000000000000000072
:1050C0000348854600F0E8FC0048004759B900084D
:1050D000F81B00200448804704480047FEE7FEE72D
:1050E000FEE7FEE7FEE7FEE7059C0008C15000086A
:1050F00030B50B46014600202022012409E00D4670
:10510000D5409D4205D31D469540491B25469540F7
:1051100040191546521E002DF1DC30BDF0B51FB40C
:105120000646002082B005464024019100901BE015
:10513000019922460F46304600F098FB049A059BE1
:10514000801A994110D310461946224600F07EFB82
:10515000361A8F410197224601200021009F00F05E
:1051600075FB38184D4100902046641E0028DFDC96
:10517000019B00982946324607B0F0BD03460B4319
:105180009B0703D009E008C9121F08C0042AFAD2FD
:1051900003E00B780370401C491C521EF9D2704783
:1051A000D2B201E00270401C491EFBD270470022BF
:1051B000F6E710B513460A4604461946FFF7F0FF16
:1051C000204610BD30B504460020034600E05B1CBD
:1051D000934203D2E05CCD5C401BF8D030BDF8B503
:1051E00002464A40D40F42004B0052085B089A42E4
:1051F00002D20246084611464A0023D0C30D4A0097
:10520000DDB2120EAD1A202D35DA49020126490A07
:10521000F6058A19002C00D0524220214F1B11465E
:10522000B9402A411018C20D9A4221D0002C17D043
:10523000012D08DCDA05801AD20F8019D207DBB203
:1052400000F040FBF8BDDA05801A012340001B0680
:10525000C01880185A428018CA0F1043490007E04E
:105260004908C2071143DA05801A801940088018DE
:1052700000F020FBF8BD61000122511A001BF7E786
:105280000122D2075140AAE70122D2075040A6E7E7
:1052900070B502464A40D50F40004A00ED0740086D
:1052A0005208002814D0002A12D0C40DD30D410298
:1052B0000120C0055202490A520AE41A09181218BC
:1052C0007D34914201D3641C00E04900002C01DAD6
:1052D000002070BD0023914201D3891A0343400886
:1052E00049000028F7D100290AD0914202D10121BA
:1052F000C90705E0914201D2012101E00121C94322
:10530000E005C018401900F0D5FA70BD420005D084
:105310004200120E52428A4201DB00207047C9054A
:1053200008187047F0B507460846584087B0C00FC8
:10533000049048000E46590040084908BC1A8841AC
:1053400005D2384631461E4617460B4602465800DF
:10535000400810434CD0300D039040055900400DDB
:10536000490D0590401A0290402872DA1803012175
:10537000000B09050843019004980092002805D00D
:1053800001995242002088410092019002984021E8
:105390000A1A0199009800F059FA05460C466B4626
:1053A00007CB00F074FAC0197141039A0E0D002367
:1053B000D71756401A467A40164344D0049A002A1A
:1053C0002DD0029A012A039A15DC1205C01A9141C8
:1053D00001263605001C7141D20F059ED2070093AD
:1053E000019202962A46234600F0B2FA07B0F0BDB9
:1053F00038463146FAE71605224A0F46B218C01A57
:10540000B74101210905001C4F4100187F41114699
:1054100018187941E20F10436D19644113E0E20757
:105420006D0815436408C2071443039A0126120548
:10543000C01A91413605001C7141CE074008304327
:105440004908C01851412A46234600F074FACDE7B6
:10545000FFE7049801224000C117121A00238B4174
:1054600004983146C417381AA141EEE730B401243C
:10547000E407634030BC55E730B40124E4076140E1
:1054800030BC4FE70000E0FFF0B51FB488B00B99C7
:105490000998002448400999C00F4900490809911A
:1054A000C0070B990090490049080B910999089889
:1054B000A64608431CD00B990A98084318D00998AF
:1054C00001244000420D4800410D099824050003C5
:1054D000000B204309900B980003000B20430B9016
:1054E00050181C494018002201901446104605E04F
:1054F000002001460DB0F0BD032801DA034600E0AC
:1055000003239C46C11A0AAE0AE05F0008ADED5BBA
:105510004F00F75B7D430027AA187C41491C5B1EA6
:105520006145F2DD410004AB5A522104120C0A43DA
:10553000240C401C0828DFDB01980290009970467B
:1055400001910090059B049A0799069800F000FAD3
:10555000D0E700000DFCFFFFF0B50C465C4085B0C5
:10556000E40FE40703944C000026640859009446B5
:10557000490802460296224321D062460A431ED0C1
:105580006200570D4A000E032303550D0124024605
:105590002C492405781B1B0B360B4018234326434C
:1055A000614600901C46501AB44103D30098401C39
:1055B000009002E0921800985B41002803DA002076
:1055C000014605B0F0BD00200121090507468646C9
:1055D00011E064461D46141BB54106D36546521BB7
:1055E000B341744607430C43A646CD07400849081B
:1055F000284392185B4105460D43EAD110461843F3
:1056000013D06046194650407140084306D06046AA
:10561000101AB34106D20122002306E00022012322
:10562000DB0702E00122D2435310009874460105C3
:10563000381C6141029C039D0019694100F07BF90F
:10564000BFE70000FD03000070B54B005B0803439B
:105650000BD04B005C0D002633466542B341D41796
:10566000AD1AA34102DB0020014670BD12053018BF
:10567000514170BDC217C10F504010B54018CA0744
:105680009623002100F01EF910BD10B500229623CC
:10569000114600F017F910BD0EB5C217C10F5040EA
:1056A000CA0740180021054B0293019200910A4657
:1056B0000B4600F04DF903B000BD000033040000BC
:1056C0000EB505490291002100910A460B46019151
:1056D00000F03EF903B000BD330400004100400279
:1056E0000122400AD205090E80187F2901DA002024
:1056F0007047962903DC9622511AC84070479639A4
:105700008840704770B5CD0F4A0009030123090B8B
:105710001B0519430B4BED070024520D9A4201DA89
:10572000002070BD074B34339A4203DC9A1A00F014
:105730009DF802E00449511888402C43F1D04042C2
:1057400070BD0000FF030000CDFBFFFF4A0009030E
:105750000123090B1B051943094B10B5520D9A4241
:1057600001DA002010BD064B34339A4203DC9A1A4A
:1057700000F07CF810BD03495118884010BD0000AE
:10578000FF030000CDFBFFFFC20FD207400040081F
:105790000BD0C10D0723DB01C91840020905400ADF
:1057A0001143C2084007114370470020014670476B
:1057B00010B5002904DB0124E40740428C41214656
:1057C000002B04DB1C460123DB075242A3418B4222
:1057D00000D1824210BD000010B5002904DB012475
:1057E000E40740428C412146002B04DB1C46012388
:1057F000DB075242A341994200D1904210BD000004
:10580000CB0FDB07490010B5490802460A4307D011
:105810000A0D07240903E401090B121B002A01DC0D
:10582000002010BDC900440F0C43C100E018D20590
:10583000801800F03FF810BD0122D207002800DBDD
:10584000101A002900DB511A8142704710B5202A36
:1058500004DB0146203A9140002010BD91402023F6
:105860009C1A0346E3401943904010BD10B5202A0E
:1058700004DB0846203AD040002110BD0B46D3403F
:10588000D0402024A21A91400843194610BD10B5FB
:10589000202A06DBCB170846203A1041C1170B43DC
:1058A00006E00B461341D0402024A21A9140084341
:1058B000194610BD002904DA401C490001D14008F6
:1058C0004000704770B40024050C05D1102400047A
:1058D00002D1002921D01124050E01D10002083483
:1058E000050F01D10001241D850F01D18000A41CEA
:1058F000002801DB4000641C002908D020252E1B55
:105900000D46F540A14000D001212943084301067E
:105910001B1B000ADB1D02D5002070BC7047DB0595
:10592000181880180029F8DA401C4900F5D170BC1D
:1059300040084000704710B5002B08DA0024401CD6
:10594000614192185B411A4301D14008400010BDEB
:10595000F0B51FB482B005460C0003D0084604F031
:10596000F5FE02E004F0F2FE2030024600902146EF
:105970002846FFF76BFF049B059A04460F46184321
:105980001143084314D0184610431BD000984021FF
:105990000A1A18460599FFF769FF05460E46009A50
:1059A00005990498FFF752FF084305D0012004E051
:1059B0002046394607B0F0BD0020C11705430E430D
:1059C0002C43374300990E986305401A7905E40A81
:1059D00000220C43FD0A0A3002D500200146E9E707
:1059E0000105101969410C9C0D9D00196941FFF7D3
:1059F000A2FFDFE7FEB500231A461B1A8A4103DB2C
:105A00000020014603B0F0BD4A000D0301212D0B1B
:105A10000905520D0D43D10702D100186D41521EE8
:105A20005110FF31FF310131002704463E46384610
:105A3000009701910246012100200905FFF716FF9A
:105A4000C3197141F818324684468E464A41614670
:105A50002846611A904104D36046241A954176463F
:105A60001F46241900986D41401C00903428E1DD48
:105A7000F91930467041091BA84103D20022D243D4
:105A8000134601E00022134601980105381C7141BC
:105A9000FFF751FFB6E70000064C0125064E05E072
:105AA000E36807CC2B430C3C98471034B442F7D33F
:105AB000FFF70AFB40C8000860C8000870B58C18E2
:105AC0000578401C6B075B0F01D10378401C2A113D
:105AD00006D10278401C03E006780E70401C491C79
:105AE0005B1EF9D12B0705D40023521E0DD40B7079
:105AF000491CFAE70378401CCB1A921C03E01D787E
:105B00000D70491C5B1C521EF9D5A142D8D3002050
:105B100070BD000038B50446064805490068FFF727
:105B2000E7FA604300E0401E00900028FBD138BD3A
:105B300040420F0084010020F8B5044600688168E7
:105B40008907890F012902D10168C90722D181681B
:105B5000114A10261140012500290ED181682943E0
:105B600081600120FFF7D6FF01F028F807460CE01E
:105B700001F024F8C01B0A2807D9606D3043606526
:105B8000A06D2843A0650120F8BD20680068C043CF
:105B9000C007EDD10020F8BD170000801FB50B48ED
:105BA00000900B4801900B4802900B480390694607
:105BB0000A4805F0C1F90A4A08481146083905F0B3
:105BC000A9F800F06FFA002004B010BD49C6000823
:105BD00025C6000885C6000883C60008900100207D
:105BE0001000002010B500231A4603E0845CE3187F
:105BF0009BB2521C8A42F9D3D84380B210BD000038
:105C000010B5034800F096FD024800F093FD10BD6A
:105C1000981700205017002030B5446C1C252C40EC
:105C20000125A540046C6560046863608368102BDF
:105C3000036803D099600068C26030BD9A60006854
:105C4000C16030BD1449012048720A4602205E320C
:105C5000507203203C3A507204200E3A50720F48A2
:105C60000D4B0078087022310870203108770C49FC
:105C70005A1C0878587149789971233318715971F1
:105C8000203318775977107551751A461E321075E2
:105C90005175107651767047E81100203E010020C2
:105CA0006001002010B503F097FE202003F052FFA2
:105CB000012005F0ABFB002003F04CFF044805F089
:105CC00049FA044805F0F8FC002005F02DFD10BD50
:105CD0000001002083800000F8B503F049FF052093
:105CE0000121000700F056FF0025144C002800D0C9
:105CF0006560134E0221304600F04CFF002815D19C
:105D0000012020700F48808F00280ED00127BF028D
:105D100000223946304600F04AFF0A2004F06AFFAC
:105D200001223946304600F042FF6560012000F054
:105D300069FE022000F066FEF8BD00007001002040
:105D400000040050E80D00207047000010B508491D
:105D500000224A6107494B684C1523434B604B684E
:105D6000082423434B60C009C001026010BD00003D
:105D7000E0170020002002407FB500250C460646B3
:105D8000039500F00FFEE009029003A9019600952B
:105D9000684600F09FFD002804D000F0D7FD0020E9
:105DA00004B070BD00F0D2FD0120F9E710B500236A
:105DB00002E0C45CCC545B1C9342FAD310BD0000DB
:105DC00010B5214A00219069C305204804D54169D6
:105DD000022319434161911593699B0505D54369D8
:105DE0000124234343616302194393695B0505D58D
:105DF0004369082423434361E301194393691B0565
:105E000005D543690424234343616302194393691D
:105E10009B0405D54369102423434361630219435E
:105E200093699B0304D5446920231C4344611943AF
:105E30009369DB0305D54369402423434361A002F2
:105E40000143916110BD000000200240E0170020D6
:105E500070B5054600F0B2FE0646184C0AE0681C14
:105E600008D0002D04D000F0A9FE801BA84201D963
:105E7000032070BDA069C007F1D1A069800701D5DA
:105E80000220A061A069C00511D4A06980050ED4CC
:105E9000A06940050BD4A069000508D4A06980045E
:105EA00005D4A069800302D4A069C00303D5FFF71D
:105EB00087FF012070BD002070BD0000002002405F
:105EC000F8B51746002605460C4600F06BFD09E0C4
:105ED00029460220226800F047FD002804D1241D35
:105EE0002D1D361DBE42F3D300F030FDBE4201D25F
:105EF0000020F8BD0120F8BD10B508490246002079
:105F0000054B497905E044001C5B944203D0401CDA
:105F1000C0B28842F7D310BD8C130020700000205F
:105F200010B500F03CFE10BD10B5094801F05CF85A
:105F300080B2FFF7C5FB074A074BFFF7A5FA00221F
:105F4000064BFFF709FBFFF701FC80B210BD000014
:105F500004160020F853E3A59B843E4000408F4088
:105F600070B50024204603F0B7F947494748A2001E
:105F7000641CE4B28150142CF9D3464944480A7990
:105F800002754979417544490A7802764978417623
:105F90003F490520133148720A2005F07DFB7D2022
:105FA000400105F093FB3A49002213310C2005F023
:105FB0005DFC00210C2005F06BFC384801F014F862
:105FC000344C0125203CE084AD0309E0334801F066
:105FD0000BF880B2E084A18EFF392D39884206DBB0
:105FE000A18E80B28842F1D349198842EED80220AE
:105FF00005F0A2FB002003F06FF9294D00210F20CE
:1060000005F0CAFA2842E063F8D0E06B411C38D0B2
:10601000400435D58122D20100210F2005F0FBFB81
:106020000021102005F0B8FA41061948490E002257
:10603000C73005F0E7FA164DC735687A05281FD135
:1060400002221549681DFFF7BDF8002818D1114834
:10605000AE7C66710422691C3430FFF78FF8294644
:106060001331084672000D466930FFF787F86079F2
:106070002946420005484838FFF780F80320207081
:1060800070BD04F0D7FB0000FFFF0100EC130020FF
:10609000491200209000002060010020041600201A
:1060A00000D0272410B5144C144822461032114653
:1060B000083904F02FFE0022114BE168A068FFF7B9
:1060C0004BFA104A104B05F04FFD00220F4BFFF723
:1060D000D3F900220E4BFFF7D7F9FFF791FB2060B1
:1060E00000221346E168A068FFF762FB01D0206838
:1060F00010BD0020206010BD000000209001002095
:1061000000AA8F406C45D9CC955BC83F0000F03F9A
:1061100040A5E54010B5084800F096FA0A21064867
:1061200000F032FA044800F01DF9800503D502485A
:1061300000F01AF980B210BDA8150020F8B52F4D57
:1061400000220121284600F032FDFFF7E3FFFFF7B0
:106150009CFA2B4E3146FFF79BF82A4C0122A06097
:106160001146284600F023FD2749A06800258842F3
:106170003EDB2078254F002815D02570FFF7CAFF99
:10618000FFF783FA3146FFF783F8A060FFF7FCFAC8
:1061900000223B46FFF76AF900221D4BFFF774F916
:1061A000FFF72EFB6060A068FFF7EEFA00223B4687
:1061B000FFF75CF9174A184BFFF766F906460F46DA
:1061C0006068FFF7E1FA134A144B5242FFF75CF99B
:1061D00032463B46FFF7A6F8FFF712FB1049606016
:1061E000884201DD616004E0FF21C905C84200D397
:1061F00065606068FFF772FAC0B2F8BD0004005035
:1062000000401B44480000200000604000000C409B
:1062100000E064403333333333B33040CCCCEC3F15
:106220000000C842F8B5054604464035287C0026E3
:10623000012808D001202874206881688907890F07
:1062400001290ED101E00220F8BD0168C90708D07C
:10625000606D2021084360650126002028743046C7
:10626000F8BD616DFF220132914302221143616545
:10627000C1688907890F0091C16889088900C160D8
:106280002068816892071143816000F097FC0746FF
:106290000EE000F093FCC01B0A2809D9606D0221B2
:1062A0008843102108436065002028740120F8BD50
:1062B000206880680028ECDB2068C168009A1143E0
:1062C000C160606D80088000401C6065C5E700000B
:1062D000F8B506460D464036317C01290DD0012126
:1062E000317401688A68520709D5416D2022114333
:1062F0004165002030740120F8BD0220F8BD174B25
:106300006A68D80547109A42154C8A6A2B6812D0E1
:106310005B035B0B1A438A622968490305D5A168B0
:106320000143A1600A20FFF7F5FB2868800312D51E
:10633000A06838430EE05B035B0B9A438A622968CE
:10634000490302D5A1688143A1602868800302D572
:10635000A068B843A06000203074F8BD01100000B0
:1063600000270140406D70470068006C70470000D6
:1063700070B5040006D0606D264600254036002822
:1063800002D006E0012070BDA5653574204600F0FE
:10639000D3F8606DC00603D421688868400705D52E
:1063A000606D1021084360653574EBE7606DFF2276
:1063B0000132904302221043606588688207920F81
:1063C0005B48012A02D10A68D2072BD103236268F5
:1063D0009B079A4205D05B429A4202D05B009A42E8
:1063E00009D10A69920092080A6121680A69636802
:1063F0001A430A610CE00A69920092080A618168F6
:106400000F22920491438160816862681143816028
:106410002168CA6818239A43CA602168CA68A368B9
:106420001A43CA60816801225206914381608168E3
:10643000A28E52061143816020688168C90004D48D
:10644000816801221207114381602068C168394ABE
:106450001140C1602069E168022825D00020014375
:10646000204620300278037B52035B001A4311431D
:10647000226B1143A26992031143E269D2031143D3
:106480002268D3681943D160616A0A46FF3AC23A6A
:1064900005D0A26A11432268D3681943D1604278BB
:1064A0000121012A02D00BE00420D8E7007800285F
:1064B00023D0606D202210436065A06D0843A06565
:1064C000E06B012820681FD00169C90703D001696A
:1064D00049084900016120684169C908C900416152
:1064E00020684169A26B11434161A565606D800818
:1064F0008000401C6065002070BD2068C2680123D8
:106500001B041A43C260DBE70269FF239B009A4326
:10651000026120680269236CA66C1A43636C3343E2
:106520001A430261206802690A430261D3E700004E
:10653000002701401902FEFF10B586B00446142161
:106540006846FEF734FE0E492068884216D10D4891
:10655000416B421511434163C16A01221143C1627B
:10656000C06A694610400590022000900320019007
:10657000002002900520000700F050FA06B010BD80
:106580000024014000100240F8B504464069254649
:1065900040350E4608280BD02068C068C00709D0D7
:1065A000606D202108436065002028740120F8BD3B
:1065B000082700E00C2700F001FB009011E0701CA0
:1065C0000FD0002E05D000F0F9FA0099401AB04221
:1065D00007D9606D042108436065002028740320FA
:1065E000F8BD206800683842E9D0606D0121490299
:1065F000084360652068C16809058A0F0C21002ADC
:106600001BD12022125D002A17D10268120714D56F
:10661000826853070122002B08DB43688B434360E9
:10662000606D130298431043606506E0606D20239F
:1066300018436065A06D1043A065A069002801D1D2
:10664000206801600020F8BD70B504462168002074
:106650008968490721D425464035297C01291CD069
:1066600001212974E169012904D02046FFF764FA69
:10667000002811D1616D0A4A1140FF2201321143F5
:1066800061650021A165297422681C2111602168BF
:106690008A6804231A438A6070BD022070BD00001E
:1066A000FEF1FFFF30B5014620314A790023022A6E
:1066B00004D00422C2630B71012030BD026814684B
:1066C0000E25AC431460026814686408640014600A
:1066D000446C1C22144001221546006CA540456004
:1066E0004A7118460B7130BD70B500240146203147
:1066F0004A79022A03D00421C163012418E0026808
:1067000013680E25AB431360026813685B085B00D7
:106710001360436C1C221340012215469D40036CFC
:106720005D604A7100220A71816B002900D08847A0
:10673000204670BDF0B4016C0D6801680C68466CB1
:106740001C2304221E401746B7402F420ED0670775
:106750000CD50C68A40602D40C6894430C60416C00
:1067600019408A40016C4A60016B1AE00227B74069
:1067700002462F402032002F17D0A70715D50C68EE
:10678000A40605D40C680A25AC430C6001215171A4
:10679000446C02211C40036CA1405960002111711E
:1067A000C16A002918D0F0BC08470827B7402F421B
:1067B00012D0240710D50C680E25AC430C60446C35
:1067C00001211C400B46A340046C6360C1635171FE
:1067D00000211171416BE4E7F0BC704770B5040013
:1067E0003CD01F48256814212818FEF781FC800042
:1067F00060641C482064022120462030024641711A
:1068000029681948E3680140A0686669184323694C
:1068100033431843A3691843E3691843236A1843B1
:10682000084328600121A0688903884210D00D48E0
:106830008030836A656C1C210D400F26AE40B34347
:106840008362656C63680D40816AAB400B43836271
:106850000020E06301215171107170BD012070BDF5
:10686000F8FFFDBF000002400F80FFFFF8B50446AF
:106870008C46203001790025012909D001260671B6
:1068800041790027012905D0077102252846F8BD66
:106890000220F8BD02214171E763206801684908C0
:1068A0004900016061462046FFF7B6F9206B0028D9
:1068B0002068016801D00E2205E0042291430160A6
:1068C000206801680A221143016020680168314391
:1068D0000160DBE7F8B51A4E0546307C0F4601280B
:1068E00007D0012030741748FFF7B2FA010002D038
:1068F00021E00220F8BD0020C04338606C6814E03D
:106900002046FFF723FA0F48FFF7A2FA01460E4888
:10691000426808239A434260426843159A434260A2
:10692000002901D03C6006E08034A8686A68C00194
:106930008018A042E4D8002030740846F8BD00005A
:10694000E017002050C300000020024005484168C5
:10695000022211434160416801221143416000203D
:106960007047000000200240F8B50C4C1646207C11
:106970000F46012808D0012020740948FFF768FA63
:106980000025002802D006E00220F8BD65613E60C7
:106990000348FFF75DFA2574F8BD0000E0170020FA
:1069A00050C3000011484168C9070BD0EFF31081B4
:1069B00072B60F4AC2600F4AC26081F31088416804
:1069C000C9070ED1416889070DD5EFF3108172B662
:1069D000094A0261094A026181F310884068800710
:1069E00001D50120704700207047000000200240C0
:1069F000EFCDAB8905040302BFAE9D8C16151413B1
:106A00007047000010B504494A69024202D048614B
:106A1000FFF7F6FF10BD000000040140FCB50023A5
:106A20000124A2E027462A469F403A406FD04D6895
:106A3000012D05D0022D03D0112D01D0122D16D11C
:106A400085680326AC465D00AE46AE406546B5435C
:106A5000AC46CE687546AE4065462E4386604668B5
:106A60000D79BE43ED06ED0F9D4035434560C66888
:106A70005F000325BD40AE46AE4335468E68BE403E
:106A80002E43C6604E68022E01D0122E14D1DE08AD
:106A9000B60036180196366A5D07B446EE0E0F252D
:106AA000B54000966646AE43B4460D69009EB540BB
:106AB00066462E43019D2E6206687546AE430D79EB
:106AC000AD07AD0FBD40354305604D68ED004BD5BA
:106AD000294D6E6B26436E639E08284DB6007519CE
:106AE000AC46AD689E07360F0F27B740BD4305275C
:106AF0003F07B84201D1002715E0214FB84201D12C
:106B0000012710E01F4FB84202D102270BE02BE013
:106B10001D4FB84201D1032705E01C4FB84201D1F7
:106B2000052700E00627B7402F436546AF60184DA4
:106B30002E684F689643FF0300D516432E606E689B
:106B40004F689643BF0300D516436E60AE684F682A
:106B50009643FF0200D51643AE60EE684F68964339
:106B6000BF0200D51643EE605B1C0A681546DA408A
:106B700000D057E7FCBD00000010024000000140BB
:106B80000004005000080050000C0050001C005091
:106B9000000401400069084000D0012070474269AC
:106BA00013460B401B0491430B4383617047002A3B
:106BB00001D08161704781627047000001488068A0
:106BC0007047000078010020024881680278891827
:106BD000816070477801002010B5084800240168E2
:106BE000402211430160204600F00AF8002801D03D
:106BF000012401E000F042FA204610BD00200240CE
:106C000070B504460D4D7D202978C000FEF770FA5E
:106C100001460B480068FEF76BFA00F02BFF0028D6
:106C200009D1042C07D200222146401E00F04EFA62
:106C300000206C6070BD012070BD00007801002054
:106C40008401002070477047F8B502F091FF604C56
:106C50000120E070208AFEF718FD01467F20C00564
:106C6000FEF716FB5B4D06462968FEF7B8FA28606A
:106C70000120A16AC005814201DA084603E03046DE
:106C8000FEF702FBA062FF21C9050025C84200D320
:106C9000A562607800280BD102214F48FFF77AFFE8
:106CA00002004E494E4817D00022FFF780FFE562F0
:106CB00002214948FFF76EFF4A4E002855D0E56291
:106CC000B08AFEF7E2FC434F3968FEF7B5FD5FD2AC
:106CD0004549012008705DE00122D1034048FFF7DB
:106CE00066FF208AFEF7D1FC01467F20C005FEF733
:106CF000CFFAE16AFEF773FA3C49E0628842D7DDD9
:106D000038480127F926403000900A213046FEF726
:106D1000EFF9002903D131493148FFF701F9022188
:106D20002D48FFF737FF002801D0002701E0002F92
:106D300012D102212848FFF72DFF00280CD104F0C2
:106D4000DBFE00990120888005F032FC642003F00E
:106D500051FF28492648C8600A2003F04BFF3046FF
:106D6000761EF6B20028D0D1A2E7208AFEF78DFC6D
:106D700001467F20C005FEF78BFAE16AFEF72FFA85
:106D80001D49E06288429BDB1A491948C86097E7B1
:106D900015480570708F401EFEF76CFC3968FEF7D1
:106DA0004BFD06D82079002803D014490120087033
:106DB00001E012480570708FFEF767FC3968FEF736
:106DC0003BFD04D22079002801D004F059FEF8BD23
:106DD0003C010020740100200004005000800000ED
:106DE00000000050E80D0020760000200000404028
:106DF0000400FA0500ED00E00000A0408300002040
:106E0000704770B5040010D0022025462035A873C5
:106E1000204601F0DDFCA87B032805D0204600F0C9
:106E2000B9F80020A873687370BD012070BD704769
:106E3000704710B5044600680168C943C90708D106
:106E40008168C943C90704D1012141602046FFF789
:106E5000FBFE20680168C943890708D48168C943DB
:106E6000890704D4022141602046FFF7EBFE206829
:106E70000168C943490708D48168C943490704D454
:106E800004214160204600F0F7F820680168C943FA
:106E9000090708D48168C943090704D4082141605F
:106EA0002046FFF7ADFF20680168C943C90608D432
:106EB0008168C943C90604D4102141602046FFF708
:106EC000C2FE20680168C943890608D48168C943A5
:106ED000890604D4202141602046FFF7A9FF2068DD
:106EE0000168C943490608D48168C943490604D4E6
:106EF000402141602046FFF79AFF10BDF8B504001D
:106F000005D025462035A87B002802D006E00120C8
:106F1000F8BD00206873204600F04EF80220A873E8
:106F20002068C26884466368012B01D10620824331
:106F300016486169814202D0072040038243002B3A
:106F400001D1D82082431248A66802401846304337
:106F5000676A266A3E433043A66A30431043002BDB
:106F600002D0012B04D005E02369E2691A4300E056
:106F7000E2681043054A914202D0A26911430843D6
:106F80006146C8600120A8730020F8BDFFFF000023
:106F9000F8F119FF10B500680549884207D1054886
:106FA000816B4900490881630D2000F073F810BD22
:106FB000007C00400010024010B50068084988427B
:106FC0000CD10848816BC204114381630022012166
:106FD0000D2000F07BF80D2000F06CF810BD0000D3
:106FE000007C0040001002400068C069704700004B
:106FF000F8B504460220254620351746A8731D48DB
:107000000268C3041A4302602068C2689B121A43D4
:10701000C2602068026901263243026122681020A2
:107020005060206881611021204601F041FC032856
:107030001FD0216808204860206847610821204649
:1070400001F036FC032814D0204601F0C1FBA87BD8
:1070500003280ED02068816831438160206801696F
:107060003143016120680169042211430161AE735B
:107070000020F8BD00040140704700000448416B47
:10708000012211434163816B020411438163704704
:1070900000100240002809DBC106C90E012088400B
:1070A00003490860BFF34F8FBFF36F8F7047000035
:1070B00080E100E0002805DBC106C90E0120884000
:1070C000014908607047000000E100E010B503F0DE
:1070D0008FFB10BD02494A6882434A607047000036
:1070E000007000400248016882151143016070473A
:1070F0000070004002494A6802434A60704700003D
:1071000000700040054801680222114301600448F4
:10711000016904221143016130BF704700700040D3
:1071200000ED00E0F0B5154A1368154D54152D6AB1
:107130002340ED07ED0F002B04D0002D02D0166880
:10714000A64316601668B608B600064316600D48DA
:10715000076904263743076101290DD040BF20BFCE
:1071600020BF0169B1430161002B04D0002D02D082
:10717000106820431060F0BD30BFF2E7007000409F
:107180000000014000ED00E0F8B50446007800275B
:10719000534D800671D5524E403EB06BC00004D4B2
:1071A000B06BA9050843B06301274E480168C905C3
:1071B00011D40168821511430160FFF7FFFC0090B4
:1071C00005E0FFF7FBFC0099401A642837D84548D2
:1071D0000068C005F5D532680321090560680A40DA
:1071E0000140914208D08103890F032904D13168FD
:1071F000890301D50120F8BD2A69032109040A4049
:1072000022D0084090421FD0207880061CD52869E3
:107210002A6988430121C9040A432A612A698A43E9
:107220002A612861C0050FD5FFF7C8FC009008E06F
:10723000FFF7C4FC0099411A2B48814201D9032071
:10724000F8BD28698005F3D561688803800F03289D
:1072500005D132680005824301400A433260286943
:10726000032261681204114008432861002F04D0F2
:10727000B16B012000078143B1632078C00705D0BE
:10728000E868A168800880000843E86020788007EB
:1072900005D5E8680C218843E1680843E860207858
:1072A000400706D5E868032189028843216908431D
:1072B000E8602078000706D5E868032109038843C1
:1072C00061690843E8602078000606D5E868032174
:1072D00089048843A1690843E8600020F8BD0000E4
:1072E000401002400070004088130000F8B50E46C0
:1072F000050038D05E480068C007C00FB04214D205
:107300005B4C20684008400030432060FFF756FC8B
:10731000074605E0FFF752FCC11B564881427AD868
:107320002068C007C00FB042F4D12878524C8007C3
:1073300005D5E068F0218843A9680843E060287813
:10734000C00752D06868022806D0032807D02168F9
:1073500001280AD0890504E02168890301E0216839
:107360008901002903DB0120F8BD4907F9E7E1683D
:10737000890889000143E160FFF720FC074668683F
:1073800002280AD0032814D001281ED029E0FFF7D4
:1073900015FCC11B374881423DD8E0680007800FCB
:1073A0000228F4D121E0FFF709FCC11B31488142DA
:1073B00031D8E0680007800F0328F4D115E0FFF70B
:1073C000FDFBC11B2B48814225D8E0680007800FD8
:1073D0000128F4D109E0FFF7F1FBC11B25488142E8
:1073E00019D8E0680007800FF5D121480168C90766
:1073F000C90FB14217D901684908490031430160FA
:10740000FFF7DCFB074608E005E0FFF7D7FBC11BF1
:107410001848814201D90320F8BD15480068C0070B
:10742000C00FB042F1D12878400706D5E0680721A7
:1074300009028843E9680843E0602878000707D517
:10744000E0680721C90288432969C9000843E06050
:1074500000F03AF8E168094A0906090F515CC84092
:107460000749086007480068FFF7CAFBF8BD00003D
:107470000020024088130000001002408AC7000864
:10748000840100207C010020044805490068C96887
:10749000044A4905490F515CC840704784010020E7
:1074A00000100240A3C70008044805490068C968E5
:1074B000044A8904490F515CC84070478401002088
:1074C00000100240A3C7000870B51A4AD3681A49D1
:1074D0000C2018408D0004280CD04E00082810D035
:1074E0000C2810D050680004410F0120C003491C33
:1074F000884070BD1068C00601D5084670BD28469A
:1075000070BD304670BD98020C4C000F205C1B0211
:107510009C0FD368641CDB0301D5314603E012687D
:10752000D20600D4294603F028F922460023FDF7AD
:10753000F5FD70BD0010024000093D009AC700082B
:10754000FEB505007ED0FE4CE7680C20E6680740DB
:107550000120000406402878C00747D0082F05D036
:107560000C2F0AD101200004864206D12068800336
:107570003CD568680028E5D038E00120696800043F
:10758000814203D121680143216011E005230122DA
:107590001B0492049942216802D111432160F1E752
:1075A0008143216021680140009120689043206060
:1075B000686800280DD0FFF701FB009005E0FFF799
:1075C000FDFA0099401A64287BD820688003F6D51C
:1075D0000CE0FFF7F3FA009005E0FFF7EFFA0099EF
:1075E000401A6428F0D820688003F6D428788007F1
:1075F00056D50923E868042F0DD00C2F01D1002E99
:1076000009D000283CD02168994301432160FFF74D
:10761000D5FA064628E02168490701D5002891D00F
:1076200061681F22120291432A69120211436160AC
:107630002168994301432160FFF746FFE16809068D
:107640000A0F00E08BE1BF49895CC840BE49086071
:10765000BE480068FFF7D4FA002873D120E0FFF796
:10766000ADFA801B0228AFD820684007F7D56068C4
:107670001F210902884329690902084360600FE05D
:107680002068400840002060FFF798FA064604E0B2
:10769000FFF794FA801B022896D820684007F7D499
:1076A0002878C00660D5002F0CD0A86900284AD0E1
:1076B0002068FF21013108432060FFF77FFA06466A
:1076C0002EE0C1E02068800502D5A8690028A6D078
:1076D0006068072149038843296A0843606060683D
:1076E000297F0002000A090608436060286A410BEE
:1076F0000120C003491C8840E16809060A0F91492E
:10770000895CC8409049086090480068FFF778FAA3
:10771000002817D128E0FFF751FA801B0228A2D8D1
:1077200020688005F7D56068072149038843296AE6
:10773000084360606068297F0002000A0906084368
:10774000606011E0E2E02168FF20013081432160A8
:10775000FFF734FA064604E0FFF730FA801B0228F0
:1077600072D820688005F7D42878794E000724D590
:1077700068690028306910D0012108433061FFF7A3
:107780001DFA009005E0FFF719FA0099401A022847
:107790005AD830698007F6D50FE0400840003061C4
:1077A000FFF70CFA009005E0FFF708FA0099401A7D
:1077B000022849D830698007F6D42878400766D572
:1077C00000200290A06BC00006D4A06B0121090725
:1077D0000843A063012002905E480168C90511D4E6
:1077E0000168821511430160FFF7E8F9009005E098
:1077F000FFF7E4F90099401A642825D85548006835
:10780000C005F5D5FF20AA680130824203D1316955
:107810000143316111E001218902002A07D00523CB
:107820001B029A4203D132690A433261EFE732699F
:1078300082433261306988433061A868002810D0E3
:10784000FFF7BCF9009008E05FE0FFF7B7F90146E9
:107850000098091A4048814257D830698005F4D50C
:107860000DE0FFF7ABF9009006E0FFF7A7F90099EC
:10787000411A3948814248D830698005F5D40298C8
:10788000002804D0A06B012109078843A063686A1F
:10789000002866D00C2F3ED001263606022820682C
:1078A00005D0B0432060FFF789F905462FE0B043CB
:1078B0002060FFF783F9074604E0FFF77FF9C01B5C
:1078C000022822D820688001F7D4E96AA86AE26811
:1078D0000843296BFD231B049A4311430843E060CE
:1078E000206830432060FFF769F9054604E0FFF7A0
:1078F00065F9401B022808D820688001F7D530E0E0
:10790000FFF75CF9401B022801D90320FEBD206867
:107910008001F5D425E00128F8D0E06801210904B0
:10792000AA6A014091421AD10F218904EA6A0140F2
:10793000914214D1032189050840296B88420DE04A
:10794000001002408AC70008840100207C0100204A
:1079500040100240007000408813000001D0012058
:10796000FEBD0020FEBDF8B504000ED0FF27606A02
:107970000537002500280AD0256165612646403676
:10798000A562707C002807D00AE00120F8BD60687D
:10799000B842F3D0E561F1E73574204600F03EF8D7
:1079A000022171742068026840239A4302602123F7
:1079B000A26860689B021A4038401043E3688A025C
:1079C0001340184323690B40217D1843C907C90F91
:1079D0000843A169931019400843E169382319400D
:1079E0000843216A802319400843A16A9300194083
:1079F000084321680860A0690421000C0840616AFE
:107A0000102319400843216848602068C1699143E8
:107A1000C1616565012070740020F8BD10B586B0A5
:107A2000044614216846FDF7C2FB104920688842CD
:107A300019D10F48416B821411434163C16A01227D
:107A40001143C162C06A002110400590E0200090FF
:107A500002200190032003900291049105206946C1
:107A60000007FEF7DBFF06B010BD0000003001404C
:107A700000100240094910B5401E884201D901207A
:107A800010BD074C60610321081F02F0B1FE002009
:107A9000A06107202061002010BD0000FFFFFF0053
:107AA00000E000E0F0B502462032137E012B1ED02C
:107AB000012515760223537606687468B36870272B
:107AC000BC430F68274377600068AC07A04205D02D
:107AD000084CA04202D0084CA04204D1802449683E
:107AE000A34319438160557600201076F0BD022033
:107AF000F0BD0000000801400014014070B5050011
:107B000005D02C462034607E002802D006E00120FB
:107B100070BD00202076284600F010F80220607624
:107B2000291D286802F09AF80120A077A076E07657
:107B3000207760776076002070BD0000006801212A
:107B40008907884204D10348816B01221143816374
:107B50007047000000100240F8B505460446203585
:107B6000287E012817D001262E760220687622680A
:107B700090687727FF23B8431B02984390600A68F8
:107B8000502A31D00EDC202A4BD006DC002A48D007
:107B9000102A3AD145E00220F8BD302A41D0402ACF
:107BA00033D136E0602A27D0702A12D0012000039A
:107BB000121A2AD0824228D1CB684A688968206884
:107BC00002F085F8206881680122920311438160E8
:107BD0001BE0CB684A688968206802F078F8216861
:107BE00088683843886010E0CA684968206802F0F5
:107BF000E8F85021206806E0CA684968206802F069
:107C0000F1F86021206802F06DF86E760020287689
:107C1000F8BDCA684968206802F0D3F8402120689E
:107C2000F1E711462068EEE710B586B0044614214E
:107C30006846FDF7BCFA012120688907884212D105
:107C40000A49CA6A02200243CA62C96A0190014015
:107C5000059141020091002102910391049069462F
:107C60000348FEF7DBFE06B010BD00000010024026
:107C700000040050F8B5064604462036307E0D4616
:107C800001280BD0012008273076002A08D0042ACA
:107C900016D0082A2AD00C2A4DD137E00220F8BD90
:107CA000206802F027F820688169394381612068E3
:107CB000816904229143816120688169EA6812E048
:107CC000206802F02FF8206881690122D202114356
:107CD000816120688269012189028A43826120686A
:107CE0008169EA6812021143816124E0206802F090
:107CF00032F82068C1693943C1612068C169042232
:107D00009143C1612068C169EA6812E0206802F00D
:107D10003DF82068C1690122D2021143C161206887
:107D2000C269012189028A43C2612068C169EA6887
:107D300012021143C16100203076F8BD70B5050014
:107D400005D02C462034607E002802D006E00120B9
:107D500070BD00202076284600F00FF802206076E3
:107D6000291D286801F07AFF0120A077A076E0762F
:107D7000207760776076002070BD704770B505464B
:107D80002C4602202034002908D004290BD00829D1
:107D90000ED0627F012A10D0012070BDA27E012A80
:107DA000FAD1A0760AE0E27E012AF5D1E07605E07C
:107DB000227F012AF0D1207700E060770122286835
:107DC00001F078FF0122286892070121904205D036
:107DD000074A904202D0074A904204D18268520773
:107DE000520F062A02D002680A430260002070BDCA
:107DF000000801400014014070B504460D460068BB
:107E0000002201F057FF2068016A0C4A114203D199
:107E1000016849084900016001202034002D06D086
:107E2000042D06D0082D06D06077002070BDA07606
:107E3000FBE7E076F9E72077F7E700001111000093
:107E40007047704770470000F8B502680446D06973
:107E500011689668814B05461D402023002D6CD08B
:107E6000F7077F4DFF0FBC460D402F4379D02546C5
:107E7000C7078035002F06D0CF0504D5012717622C
:107E80002A683A432A60820708D5F20706D0276895
:107E900002223A622A6804273A432A60420708D538
:107EA000F20706D02668042232622A68022632438C
:107EB0002A6002070AD50A461A406646324305D0B0
:107EC0002668082232622E6816432E60020508D505
:107ED0004A0106D501222668D20232622A681A4374
:107EE0002A602A68002A30D0800606D5880604D584
:107EF000616E002901D0204688472868216889687A
:107F0000490602D42821084225D0204602F081F9F2
:107F100020688168490619D5826840218A438260B9
:107F2000206F002812D04F498163206FFEF7DCFBE1
:107F300000280AD0206F816B06E0850611D58D06DA
:107F40000FD5616E77E020468847F8BD2046FFF7E1
:107F500079FFF8BD05E02046FFF774FF0020286098
:107F6000F7E7256E012D56D1C50654D5CD0652D55D
:107F7000102616622068816825464906403500298A
:107F80002ADA226F116849680904090CE1D02F8BA5
:107F90008F42DED9698311680968890617D40168A0
:107FA000320191430160206881684908490081607D
:107FB00020688168402291438160E3670020206649
:107FC00020680168B1430160206FFEF76BFB288BCE
:107FD000698B401A81B21AE0298B6A8B891A6A8BE5
:107FE00089B2002AB5D00029B3D00268FF25213517
:107FF000AA43026020688268520852008260E367E8
:1080000000202066606620680268B2430260204655
:10801000FFF716FF9DE7C50208D5750206D50120BA
:10802000000510622046FFF70CFF92E7050605D514
:108030000D0603D5A16E002985D18AE7400688D5B3
:10804000480686D5116820464024A1431160836705
:108050000021816600F043F97BE700000F08000073
:108060002001000439A1000810B5040003D0A06F5E
:10807000002802D007E0012010BD00217420015526
:10808000204600F027F82420A067206801684908EE
:1080900049000160204602F00FF90128ECD0606A27
:1080A000002802D0204601F031FF206841680922F3
:1080B000D20291434160206881682A229143816005
:1080C00020680168012211430160204601F084FF0D
:1080D00010BD0000F0B587B0064614216846FDF7D4
:1080E00066F82C493068884251D12B48416B0122F7
:1080F000920311434163C16A01221143C162C06A04
:108100000025104005900320400200900220032724
:1081100001A9A1C104200490052069460007FEF7CB
:108120007DFC1F4C1D48A560E56081C48027E5608B
:10813000A7602020256160610002A0611848083C0A
:10814000FEF74CFB002801D0FDF7FEFD3467A66268
:10815000144C12482146143820600320606010201F
:108160000831A1C16561A561E56120462562FEF780
:1081700035FB002801D0FDF7E7FDF4660022012160
:108180001B20A662FEF7A2FF1B20FEF793FF07B09D
:10819000F0BD0000003801400010024030000240F5
:1081A000501700209817002070B5C36F202B27D1DF
:1081B00000290BD0002A09D0012483682403A3429C
:1081C00006D10369002B03D1CB0701D0012070BD7C
:1081D000034660331C7D012C12D001241C75002342
:1081E0000366084C0368A34207D05C68240204D5E8
:1081F0001C680125AD062C431C6002F05DF970BDC2
:10820000022070BD0048004070477047FFB504462B
:10821000806F83B017460D4620285ED1002D0AD00E
:10822000002F08D0A168C001814207D12069002831
:1082300004D1E80702D0012007B0F0BD204660302D
:108240000090007D012848D0009801210175002090
:10825000802108512120A067FEF7B0FC2646403659
:108260000190378277820120A1680003814202D108
:108270002069002805D02F460025009900200875A8
:1082800011E00027F9E700228021204602F05AF988
:10829000002815D1002F15D02168387888627F1CFE
:1082A000708A401E7082708A019B00280698009098
:1082B000E9D100224021204602F044F9002808D0EC
:1082C0000320B9E728882168C005C00D8862AD1C6D
:1082D000E6E72020A0670020AEE70220ACE7704769
:1082E000034D044C04A002F027FAE560FAE7000011
:1082F0000400FA0500ED00E0486172644661756CA7
:10830000745F48616E646C65722E0D0A0000000097
:1083100000B585B014216846FCF749FF03480221E7
:10832000418300F0EFFB05B000BD00003C010020E0
:1083300010B505242407002204212046FEF737FC4F
:10834000002208212046FEF732FC0A2002F059FCE8
:10835000012204212046FEF72AFC0A2002F051FCEB
:10836000002204212046FEF722FC10BD10B5052492
:108370002407002204212046FEF719FC01220821CF
:108380002046FEF714FC0A2002F03BFC01220421E7
:108390002046FEF70CFC0A2002F033FC00220421E8
:1083A0002046FEF704FC10BDF8B50024052607465C
:1083B00025463607002204213046FEF7F8FB0A2046
:1083C00002F01FFC012204213046FEF7F0FB60069C
:1083D000040E08213046FEF7DDFB002801D0641CA6
:1083E000E4B2052002F00DFC6D1CEDB2082DE1D3C6
:1083F000002F03D0FFF79CFF2046F8BDFFF7B6FF24
:10840000FAE770B5052605463607002204213046F6
:10841000FEF7CDFB0024E80901D0012200E0002294
:1084200008213046FEF7C3FB6806050E0A2002F05D
:10843000E8FB012204213046FEF7B9FB0A2002F0D6
:10844000E0FB002204213046FEF7B1FB0A2002F0D7
:10845000D8FB641CE4B2082CDDD370BD10B5052434
:108460002407012208212046FEF7A1FB0122042156
:108470002046FEF79CFB002208212046FEF797FBD2
:108480000A2002F0BEFB002204212046FEF78FFBEB
:1084900010BD10B505242407002204212046FEF754
:1084A00086FB002208212046FEF781FB0A2002F00D
:1084B000A8FB012204212046FEF779FB01220821B6
:1084C0002046FEF774FB0A2002F09BFB10BD70B53E
:1084D00005252D070024012208212846FEF767FB09
:1084E000062002F08EFB012204212846FEF75FFBE6
:1084F000062002F086FB07E0641CE4B2FA2C03D9E4
:10850000FFF7C7FF012070BD08212846FEF742FB98
:108510000028F1D1002204212846FEF748FB002064
:1085200070BD0000F8B501F089FD01F0B9FD5B48B0
:108530000068C069FDF7F8FC594C5A49A082898F40
:10854000594E0025002931D0A26A730357499A4237
:1085500002DB02220A7000E00D700A780121890214
:10856000002A05D0012A0ED0022A10D0032A1DD1DC
:10857000608B01282ED0022818D1484808214038A5
:10858000FFF73AFC12E0FF22F5329042F0D2608B06
:1085900001281DD0022804D008E03046FEF707FB72
:1085A00004E03E4808214038FFF7E8FBFDF7C6FD30
:1085B00020700121C9023046FEF7ECFA0127FF03C3
:1085C00000282DD03A480560A079002804D007E0A3
:1085D0000022E2E70122E0E70120A07102F014F896
:1085E00080213046FEF7D6FA002806D00022082166
:1085F0003046FEF7DCFA012205E001220821304670
:10860000FEF7D5FA0022052039460007FEF7CFFA1B
:10861000244C284E4034A08C274F012803D01CE066
:10862000A5710022EAE725486946088072B68021D4
:108630002348FDF7A1FB002804D002226946204808
:10864000FDF73EFC62B61FA002F076F8A58403F0A9
:10865000AFFF642002F0CEFAFE60608C012808D1E2
:1086600010486584058003F0A3FF642002F0C2FA7D
:10867000FE60208C012806D1258403F099FF642038
:1086800002F0B8FAFE600748124A0188914202D10E
:10869000C088002800D1FE60F8BD0000CC16002084
:1086A0003C010020E80D0020000400508100002063
:1086B000740100200400FA0500ED00E0AAAA000001
:1086C000384A0008BDF8C8EBC9FDBCB6C4A3CABD92
:1086D0000D0A0000AA55000008B55721202000F01F
:1086E0006AF80321212000F066F84021222000F0E2
:1086F00062F80821232000F05EF8AA21302000F063
:108700005AF8084801210187322000F054F802216C
:10871000332000F050F8684600F006F80A2002F016
:1087200070FA08BDE80D002010B501460F2000F0DA
:1087300021F8002800D0012010BD10B50446FFF735
:108740008DFE3220FFF75DFEFFF7C1FEE0B2FFF7BE
:1087500058FEFFF7BCFEFFF781FE3320FFF751FE06
:10876000FFF7B5FE0020FFF71FFE0446FFF791FE5E
:10877000204610BD10B50C46FFF7DFFF207001202A
:1087800010BD70B50D460446FFF768FE3220FFF7B6
:1087900038FEFFF79CFEE0B2FFF733FEFFF797FECF
:1087A0002846FFF72EFEFFF792FEFFF772FE0A2023
:1087B00002F027FA70BD10B5FFF7E3FF012010BDEE
:1087C00010B50248FEF735FB10BD0000041600206E
:1087D000FEB50446002772B6334A01688B1804D1EF
:1087E0003248C76803208004074088680190C86841
:1087F000009048698E69002B08D12C4940398B6A5A
:10880000CD042B438B628B6AAB438B6201463143B1
:108810003CD025492368CB4205D12449CA680323AB
:108820009B049A43CA6025462035002810D0216851
:108830000A6901231A430A61216848610821204618
:1088400000F036F8032800D1A8732168082048609A
:10885000002E10D0206801690122114301612068B7
:1088600086611021204600F023F8032800D1A87368
:108870002168102048600C482168C14206D10B488D
:10888000C1680322920491433943C16020680169A1
:1088900049084900016121680198886021680098B1
:1088A000C86062B6FEBD00000084FFBF40100240F9
:1088B00070B506460B480D46002409490068FCF7D0
:1088C00017FC7D21C90048433168401E00D10324B4
:1088D0000B682A469A4301D00028F6D1204670BD85
:1088E000204E0000840100201CB500211648009194
:1088F000144A01910260C16312054260816007223F
:108900008263012202610246C16020321170FF239E
:108910005170C23343628162117301638161042229
:1089200041634261C161FDF723FD08480090801357
:10893000019069460448FDF7CBFC00210248FDF791
:1089400071FC1CBD00240140A81500200200000499
:1089500008B50848016B012211430163006B012136
:108960001040009000220A20FEF7B0FB0A20FEF71C
:10897000A1FB08BD00100240F0B587B01421684685
:10898000FCF715FC4748C26A04210A43C262C26A66
:108990000A400592C16A80263143C162C16A3140F2
:1089A0000591C16A01242143C162C16A2140059138
:1089B000C16A02252943C162C06A22462840059047
:1089C00005201C210007FEF7F2F80122364937483E
:1089D000FEF7EDF8002236493448FEF7E8F8912119
:1089E0000520002209020007FEF7E1F83148019056
:1089F000002705206946029700940007FEF70EF84D
:108A00000C20009011200190032003900520029774
:108A100069460007FEF702F810206A46039591C2E6
:108A2000052069460007FDF7F9FF11200190029724
:108A30006946039700941D48FDF7F0FF1E4801901A
:108A40006946009502941948FDF7E8FFE00200909E
:108A50006946019702951548FDF7E0FF17486946FA
:108A600091C1694611480397FDF7D8FF9120000294
:108A7000694691C10520694600070397FDF7CEFFBF
:108A800069460A48019700960294FDF7C7FF002245
:108A900001210520FEF71AFB0520FEF70BFB07B0AE
:108AA000F0BD000000100240010200000004005070
:108AB00008300000000011100000211008320000F2
:108AC00010B50F4C0D482060FF200530606000207D
:108AD000A060E06020616061E061012120624902E4
:108AE0006062A161A0620720E0622046FEF73BFFC2
:108AF0002068016840221143016010BD0030014030
:108B00003416002010B58AB000240494059406940D
:108B10000794089401211848099400940194029440
:108B2000890703940160092184604160046113494D
:108B30004461C160FEF7E2FF01200003049004A934
:108B40000D48FFF709F80C48FFF7F8F8089408A952
:108B500009480994FEF7A6FF60200090084801909C
:108B600002940822694603940348FFF783F80248F9
:108B7000FFF75AF80AB010BD8C16002093040000CD
:108B80005702000000B585B014216846FCF70FFBC2
:108B90000E480D490160E1214902416000218160D8
:108BA000C160016181610C22C161426101623021B9
:108BB00041620121090381634900C163FFF754FA4F
:108BC00001F01CFD05B000BD00380140CC160020AE
:108BD00070470000F0B589B00A2002F05DFD7D20ED
:108BE000400102F073FDFA4C0025A570F948E065DC
:108BF000A07B0C2801D30B20A07360790A2801D92F
:108C00000A206071F448E570F44E00783071F44940
:108C1000A079097840000843E17C89000843F0719D
:108C2000A06BF070010A3172401CA0636079B074CF
:108C300042003046EB491330FCF7A0FA6079E9496D
:108C400082004000801960311330121DFCF796FA43
:108C500060790621420048438019E3491730921C8D
:108C6000FCF78CFA2C20205E002803D0DF49098A0B
:108C70000818A0856079D649C000203182190B7B85
:108C800053764B7B937606227272D94A1D30127846
:108C9000B272628C3273D14A0B79133A13754979E7
:108CA00051750022CD4902F0E1FD60790021C0003C
:108CB0001D3002F0EDFDCF48FEF796F90127E08464
:108CC000BF0309E0CB48FEF78FF980B2E084A18EA4
:108CD000FF392D39884206DB81B2A08E8142F1D363
:108CE000C0198142EED8022002F026FD01210022A7
:108CF0000903C148FDF75BFFB8480126C571E5735C
:108D0000E57266732573BB48FEF76EF9208507464A
:108D1000E5706079FCF7D4FCB84AB94BFCF7B4FBBA
:108D200001F004FF0022B74BFCF7FCFAFCF70EFD44
:108D30000006C10CC81980B2F1036085884201D3D6
:108D4000401A6085B048A0642079401C2071A94871
:108D5000FEF74AF9E084A3489D4F643840370690F7
:108D6000B2E1A448FEF740F9E0840BE0A148FEF729
:108D70003BF980B2E084618D884203D3A34A89180D
:108D8000884207D300210F2002F006FCA049E063CF
:108D90000842EBD0E06B411C1FD040047ED58122FD
:108DA000D20100210F2002F036FD0021102002F038
:108DB000F3FB41068B48490E00227C38A16502F086
:108DC00021FC002002F082FC002002F034FC8548E7
:108DD0007C38417A0729C3D101E001F02BFD022242
:108DE0008C49401DFCF7EEF90028B9D102F0A1FD35
:108DF000E167A06702F08AFD754B803303C3E0781A
:108E00007849401CE07083390B7A68460370497AD0
:108E1000417000880390A18C88427DD16F497E48C3
:108E20008C31C98E01806D4969488C31098F01846C
:108E30007048FEF7D9F8E08402F0C0FA6448FF22D7
:108E400080300168406852040023891858410206A6
:108E5000080A10434108490000900A0E08025C49C4
:108E60008031CA6088605D48E36F0A30A26F02F00B
:108E700035FD607981005948081855491630803110
:108E80000CC902F02BFD52488030C36882685348F9
:108E9000123002F023FD0821504800E007E1417242
:108EA000B430C07C0009A07414D04E480222594945
:108EB0007738FCF787F900280CD14848E673C6716B
:108EC000A06D48491638C2B26639C81D2274FB30FD
:108ED000FCF754F960790022800040491C3002F010
:108EE000C5FC6079002180001C3002F0D1FC0098A4
:108EF00002F0CBFB012002F01FFC607202213E4811
:108F0000FDF748FE00281DD0002035490870334980
:108F10008C31488E049000E082E0B880888EF88022
:108F20008446606CFF310531A0640860DC39E06480
:108F3000C97C0907090F032900D06174A16D1C29A0
:108F400002D015E00120E0E72449214A8C31C98F85
:108F5000D185069B244A1B881380884207DD0028A0
:108F600005DD002903D0607D401C607500E065755B
:108F70002571E67204983881604678812673208CCA
:108F80002649FF30C33080B2208488420CD9494240
:108F90004018208420487D220188D200491C89B2D3
:108FA0000180914200D305801B4801887D20C000CC
:108FB0004143208C0818206500F076FD607A002877
:108FC00005D100210F2002F0E7FA0006F9D584E070
:108FD000700000203F420F003C0100205C12002086
:108FE000700100208C130020C8140020280E0020DF
:108FF0004C0100200416002000040050B81E85EB30
:1090000051B8CE3F00000840A0860100983A000009
:1090100000D02724600100206C010020E70300003D
:10902000FCF76AFF694A0321115469494A8EBA80E4
:10903000898EF980A26D1C2A06D1644B4200AC33A4
:10904000D318069A12885A808000604A604B603AB2
:1090500002905E4982189B8F138030394118626CF0
:109060004A605B498C3940185A4916300CC902F0E5
:1090700035FCE16D606C884208DA544A0299603A26
:109080005158012902D1E065039905914F49029A8F
:1090900060398958814217DD012915DD22460028F3
:1090A00012DD0398908402201070A5720CE04A4AE9
:1090B00000210F2002F0AFFB6079E178401C814273
:1090C00002D0002002F0B7FAE08C618D884200D215
:1090D00047E6424A89188842FAD8E07A012801D046
:1090E0000220E07202F06AF93B4A00210F2002F0F0
:1090F00092FB012211033A48FDF759FD207900281F
:1091000014D0384909888A008A18824200D2257012
:10911000002000F0E1F8E07B002836D02B490C312C
:109120000B7848788A78022B17D02EE0A06CE16D7E
:10913000323881420FDAE1792A4A491CC9B2E17119
:109140001288204652008A42E5D205998184022184
:109150000170A572DFE7E571DDE710280CD0C828A3
:1091600013D2214BC91C1818FCF708F803F020FA99
:10917000642001F03FFD30E61C4D28684000000EE1
:1091800003D1C878FCF781FA286000202578A37AFB
:1091900062790FE00D4E4100903E775A1836765AAC
:1091A000B74205D00A4F0225002301268C377E5294
:1091B000401CC0B29042EDD3074A2570A3728032A2
:1091C00000210F2002F027FB09B0F0BD1C14002085
:1091D000E8120020F000002000D02724983A000078
:1091E000000400504C010020E80D00206401002024
:1091F000F8B52E4C0546A06E2D4A281A411EE06691
:10920000914215D21821615E081AFCF745FA294AE5
:10921000294BFCF739F9064630200F46205EFCF753
:109220003BFA32463B46FCF77DF8FCF76BFA2086AA
:109230000020A0751D481A23C35E428C1F48008879
:1092400084461F4806881DE06046484380181D4F2D
:1092500080B23880302778436427643078431A4FCF
:109260002066C01985420BD2C8B218493022088046
:10927000206EA25E411BC91889186166A066F8BD00
:10928000491CA175A17DB142DED330204243104874
:109290006421101848430F494118A1662066302107
:1092A000401B615EC01840186066F8BD7000002069
:1092B000CF0700009A9999999999B93F5A010020CE
:1092C0004C0100206E01002078ECFFFF58010020C7
:1092D00074270000C0BDF0FFFEB5294D2988491C48
:1092E0008FB228492F800E88FCF7D6F9264A274BE3
:1092F000FCF7CAF80191009025483146FBF7F8FECB
:10930000244CE18E4218B74206D300202880224820
:10931000019E1018009D02E01046019E009DFCF782
:10932000CFF933462A46FBF7FDFFFCF70FFA6086BC
:10933000012580B2ED03A84201D3401B6086A08BBB
:10934000FCF7BEF9154A164BFCF706F90646608E87
:109350000F460090FCF7B4F932463B46FBF7E2FFBC
:10936000FCF7F4F980B2A086A84201D3401BA08686
:109370000C490098096848610098E086FEBD00002D
:10938000580100204C0100201904560E2D62404067
:10939000E17A0000700000201F050000F853E3A5EB
:1093A0009B843E400416002070470000F0B589B051
:1093B000002004900A2002F06FF97D20400102F0A5
:1093C00085F9B34800228270816BB34C491C8163DC
:1093D000B049838D098A2546C918818521460275C1
:1093E00013310791473103916D393135AB4F20303F
:1093F00005910290A64E0F21A94871710078207145
:10940000A84AB079127840001043F27C92001043D1
:10941000E071308FE070000A2072A17431461E2284
:109420009C310798FBF7AAFE402228469E49FBF78D
:10943000A5FE029903980A7BC274497B0175092035
:1094400060729A480078A072708C2073307D410061
:1094500030469C30091805980A780275497841759C
:10946000762000228C4902F001FA707906214843E7
:1094700000211C3002F00CFA022002F05DF90021FC
:109480000F2002F089F83842F063F8D0F06B411CED
:1094900018D040047ED58122D20100210F2002F095
:1094A000BAF90021102002F077F841067A48490EF7
:1094B0000022B43002F0A6F87748B430417A02298D
:1094C00002D0BDE001F0B6F902227949401DFBF758
:1094D00079FE0028F5D16E480222007D41006C48DB
:1094E0009C3009186C48B530FBF76CFE0028E8D1B9
:1094F00002F01FFA664AD167906702F007FA644AE1
:10950000803203C2049800282CD1012004906248C4
:10951000684E8C30C08E604930805D488C31098F38
:1095200001846548FDF760FD5949644AC884088C88
:10953000FF30C33080B2088490420CD95242801868
:10954000088430885D4A401C80B20B3230809042E3
:1095500001D30020308030887D22D20050430A8C15
:10956000801808654C4869468C30428E0A80808E8F
:10957000488049490422B531C81FFF38FBF7FEFD7A
:109580004348494A007D009980001150404980318C
:1095900003C900E075E0FF235B040022C0185141BD
:1095A0000906060A0E43304602F06FF871084900BA
:1095B0000A0E0802364900268031CA6088603448A5
:1095C000C36F826F3448483802F088F930488030E1
:1095D0000CC83148443802F081F92D488030C36806
:1095E00082682D48403802F079F92B49002252391F
:1095F0003C2002F03BF900213C2002F049F9012017
:1096000002F09AF82249487208468078401C887017
:1096100001210520C9030007FCF782FC1C48407AA1
:10962000002805D100210F2001F0B6FF0006F9D572
:10963000802200210F2002F0EEF81548467002E06B
:109640001349012048701248017D491CC9B20175B7
:109650000F2900D2CEE60498002810D10C4A1849F0
:10966000508C002802D00B88984201D90888508479
:10967000144980B20988401E48431349088009B044
:10968000F0BD124A00210F2002F0C5F8D8E7000013
:1096900070000020280E00205C12002000D027243B
:1096A0003C01002070010020781400204C010020B3
:1096B000600100206C01002004160020E703000078
:1096C000480100204601002044010020009027248A
:1096D000F8B531492F48086002F00EFA2F4800F023
:1096E000A3F92F4CE0822D48801C00F09DF92083C7
:1096F0002A48001D00F098F960832B4829494180D1
:10970000014640310979294F0906090E617006D1D9
:10971000C7800121C1870A21418700218187244A0E
:10972000C18E1170C18F2171818F6171817AA17099
:109730008588052165626181C6883046FBF7D8FCC3
:10974000A08101462846FBF7D3FC8800081885B2A3
:10975000164825816843FBF7B3FF164A164BFBF703
:10976000FBFEFBF7F3FFE081658231463846FBF7ED
:10977000BFFC20820146C820FBF7BAFCE083012031
:10978000A083FCF7D1FBA082E2890C490C48FDF7CD
:109790002FFCF8BD29A6000868000020004F000833
:1097A0003C01002029020000E80D0020E803000031
:1097B00018000020F853E3A59B843E40FF7F000083
:1097C00004160020F8B5754C00202071744D01205E
:1097D0002880744EC8203080207A401C2072C00738
:1097E00006D0608C411E6184022801D2C8206084AA
:1097F0000120C043FFF770FD0A2001F04DFF7D20DE
:10980000400101F063FF02216748FDF7C3F900281A
:109810003FD00020654980000978664F4900084321
:10982000634909780843B872102078726248C18889
:109830007D20C000FBF75CFC787360485E490078CF
:10984000B87338460B308A780270C97841705A492B
:10985000421C20310B7ED370497E11715649D01CB9
:1098600022310B7E5371497E9171534940310A7CFC
:109870000271497C417100223946172001F0F6FF40
:109880000021172002F004F8022001F055FF4C4F90
:1098900003E00120BEE7FEF745FE00210F2001F0A6
:1098A0007BFE3842E063F6D0E06B411C73D040048D
:1098B0006FD58122D20100210F2001F0ACFF0021E1
:1098C000102001F069FE41063A48490E0022B430EA
:1098D000A16501F097FE374FB437787A112858D137
:1098E00002223849781DFBF76DFC002851D1F81F82
:1098F000027A69460A70407A4870B97A2980C8208D
:10990000FBF7F6FB3080387B608438462E4D2838D4
:10991000C08E2880394621482839098F01842B4878
:10992000FDF762FBE084208C2949FF30C33080B210
:10993000208488420CD94942401820842888244930
:10994000401C80B20B312880884201D3002028803F
:1099500028887D21C9004843218C4018206500F0EB
:10996000A3F868460088A0841249B87CC7316071AA
:10997000420008460D466930FBF700FC6079294635
:1099800042001448FBF7FAFB608CFF2801D003204B
:109990002070F8BDFFE700F04DFF000070000020D0
:1099A0004C0100205A01002000040050400100201A
:1099B000410100205C120020E80D0020180000206A
:1099C00000D02724600100206C0100200416002034
:1099D000E7030000A413002070B586B01421684688
:1099E000FBF7E5FB01250F4EED030022294630462B
:1099F000FDF7DDF8012000240190029469460095EE
:109A000003943046FDF70AF803200190029469465A
:109A1000009503943046FDF701F8022001F0EAF8C2
:109A200006B070BD00040050008870477047000009
:109A3000F8B5044600206A461080194D55222A7058
:109A4000AA226A700322AA70661DEE702A716971DB
:109A5000144A49008918AC712246E81DFBF78EFBB9
:109A6000002007E029186A468978128889186A4612
:109A70001180401CB042F5DB611DA81CFCF7B2F858
:109A800001466846018029190078C8716846407807
:109A9000087221460931024800F0DCFBF8BD0000E5
:109AA00042150020E80D0020FEB5FFF7A1FB254878
:109AB000FDF79AFA244C86B2E68460790A21081AE6
:109AC000C000FBF7E9FD07460191606EFBF7F8FD6A
:109AD0001E4A1F4BFBF740FD00900D463046FBF73A
:109AE000EFFD2B46009AFBF71DFC3A46019BFBF766
:109AF00019FCFBF72BFE85B26586A08BFBF7E0FD1A
:109B0000124A134BFBF728FD06460F462846FBF783
:109B1000D7FD32463B46FBF705FCFBF717FE81B24B
:109B20000120C003A186814201D3091AA186854282
:109B300001D3281A60860349608E09684861E0866F
:109B4000FEBD00000416002070000020F853E3A5BD
:109B50009B843E40034A1168382389B299430143EC
:109B6000116070470030014010B5FDF72DF810BDB1
:109B700010B59AB034216846FBF719FB14210DA8E3
:109B8000FBF715FB1C2112A8FBF711FB1B48016812
:109B90000324E402A143C21489180160FDF7A2FA6C
:109BA00017480169A143016106200090FF200130A0
:109BB000029001200390102004900220099040049C
:109BC0000B90000100240C900A946846FDF7B8FC45
:109BD0000F200D9003200E900F94109401211194EA
:109BE0000DA8FDF783FB81201290032080041890BC
:109BF000149412A8FDF7C8FA1AB010BD0070004006
:109C00004010024010480168821511430160C1688C
:109C10000E4A1140C16001680D4A1140016081681F
:109C20004908490081600168012292049143016062
:109C3000C168FD2212049143C160002101610649FF
:109C40000448886070470000001002400C40FF8804
:109C5000F6FFF6FE0050000800ED00E070B5026867
:109C600001239B07114C124D984203D0A04201D012
:109C7000A84203D17026B2434E683243984203D0C3
:109C8000A04201D0A84204D103231B029A43CB680F
:109C90001A4380239A430B691A4302608A68C2629E
:109CA000096881620121416170BD00000008014026
:109CB0000014014010B5CB06DB0E0121046A994067
:109CC0008C430462016A9A401143016210BD30B5B1
:109CD0008468FF252D021B021343AC430B4323432F
:109CE000836030BD826870239A430A4307210A4388
:109CF0008260704730B5026A520852000262026AFE
:109D0000456883697024A3439C080B68A40023431F
:109D10000224A2438C68456014438361496841630F
:109D2000046230BD30B5026A10239A430262036AAE
:109D30004568826973242402A2430C6824021443F8
:109D4000202293438A68456012011A43846149685E
:109D50008163026230BD30B5026AFF2301339A434A
:109D60000262026A4568C3697024A3439C080B68B9
:109D7000A400234301246402A2438C6845602402AA
:109D80001443C3614968C163046230BD30B5026ADF
:109D900001231B039A430262036A4568C269732464
:109DA0002402A2430C682402144301225203934369
:109DB0008A68456012031A43C461496801640262FB
:109DC00030BD30B5036A046A6408640004628469C3
:109DD000F025AC43120122430A24A3430B438261C2
:109DE000036230BD30B5036A1024A3430362846963
:109DF000036A0F252D031203AC432243A024A3437F
:109E0000090119438261016230BD0000F8B51024D8
:109E100005252D07AC62AF20800000F0F2FEAC619A
:109E200001F0CEFB2F4C304F304E20670EE001F09A
:109E3000C7FB2067FEF776FB206C411C21641428C9
:109E400004D92BA000F078FC2D48C760206FB042E9
:109E5000EDD10026266420780127FF03030000F0DF
:109E6000A4FC05040C192D30320001223946284685
:109E7000FCF79DFEFFF7A6FC06E0012239462846C6
:109E8000FCF795FEFFF792FA002239462846FCF7C8
:109E90008EFE18E0A07A0122401CA07239462846A6
:109EA000FCF785FEFCF75CF8002239462846FCF7F3
:109EB0007EFEA07A052806D9267004E0FEF78AFE09
:109EC00001E0FFF773FA02210E48FCF763FE002859
:109ED00005D000200C49087001F058FAF8BD0120A7
:109EE000F8E70000700000200400FA053001CADE27
:109EF0004457204944204552524F522E0D0A00002B
:109F000000ED00E0000400507001002010B5818CCD
:109F1000C90707D001684A6801235B049A43836A32
:109F20001A434A60818C890707D501684A68012372
:109F30001B049A43C36A1A434A60818C490707D5B8
:109F400001684A6801239B049A43036B1A434A60E1
:109F5000818C090707D501684A680123DB039A430E
:109F6000436B1A434A60818CC90607D50268916821
:109F700001231B039943836B19439160818C8906EC
:109F800007D501688A6801235B039A43C36B1A43B0
:109F90008A60818C490612D503685A680121090537
:109FA000046C8A4322435A60026C8A4207D10268D9
:109FB000516803235B059943436C19435160818CBD
:109FC000090607D501684A680123DB04806C9A43BF
:109FD00002434A6010BD0000F8B5044600268030F8
:109FE0000660FCF7EBFD054620680068124F00078D
:109FF00009D501212B46002249052046009700F093
:10A00000A1FA00280DD12068006840070BD5012176
:10A010002B46002289052046009700F093FA00287D
:10A0200001D00320F8BD2020A067E06726666034D9
:10A0300026750020F8BD0000FFFFFF01F8B5154CA4
:10A04000C826E078002823D16079002820D101209B
:10A050006071114D686B0027002818D0686BC8210B
:10A06000081A0FE00D48E168405C61698847E068C4
:10A07000401CE060E068C82800DBE760696BC8202E
:10A08000401A761EE168814201D0002EEADC677139
:10A09000F8BD00005400002000000240200D002008
:10A0A00070B5224CE07800283FD1207900283CD1BF
:10A0B000012020711E4EF16900250906002933DABE
:10A0C0002156625791420AD1F06940062CD5A079F9
:10A0D000002829D0A5712089401C208124E0A17985
:10A0E000002903D1A0710A2000F08BFD002020562A
:10A0F000CC2148430F494218206912181279B262E4
:10A10000401C00222061A256CC235A438958814228
:10A110000ADC25612078401C207020780E2800D1B0
:10A120002570A078401CA070257170BD54000020DF
:10A1300000380140F801002010B5806A0022014675
:10A1400040314A834A82FDF77DFE10BD70B5846AB6
:10A15000A06FE56F2168896800260906002906DAE4
:10A16000212804D152200653204600F06BF82068C5
:10A170008068400606D5222D04D15A200653204679
:10A1800000F047F82046803001681022114301603A
:10A190002046FDF757FE70BD10B501460968806A7C
:10A1A000096889061CD400225A210A5201680A68EB
:10A1B000FF2301339A430A6001688A6852085200FB
:10A1C0008A6001688A6840239A438A602021C167B7
:10A1D000016E012904D101680A6810239A430A60BC
:10A1E000016E012902D0FEF70FF810BD5821095A5F
:10A1F000FDF726FE10BD10B5806A016E012902D060
:10A20000FEF703F810BD5821095A4908FDF718FE5A
:10A2100010BD01680A68FF2321339A430A60016870
:10A220008A68520852008A60016E012904D10168CF
:10A230000A6810239A430A602021C1670021016641
:10A240004166704701680A68C0239A430A6020216A
:10A250008167704770B5164CE278002A0CD12279DC
:10A26000002A09D10122E2700025C82903DC02225C
:10A27000A256002A01DCE57070BD0123E356CC2212
:10A2800053430C4AD1500123E356CC2673439B1809
:10A290000A460146181DFAF771FF6078401C60708D
:10A2A00060780E2800D16570A078401EA070E2E7AB
:10A2B00054000020F8010020F8B5044601688068C9
:10A2C0002369E66918436369002533431843724ADA
:10A2D0000B68724E334003430B60216848680323C8
:10A2E0001B039843E368184348602168A0699142C2
:10A2F00001D0236A18438B680B263602B34303430D
:10A300008B606749236867488B420CD1C06880071F
:10A31000800F06D0012839D0022835D0032821D15A
:10A320001EE001271FE060498B420AD1C0680C2162
:10A33000084027D0042829D0082825D00C2811D17E
:10A340000EE093420ED1C16803208002014019D073
:10A3500001208002091A19D0091A15D0814201D1B1
:10A36000082700E010274F495048403986009342A3
:10A3700032D1002F0CD0022F0DD0042F10D0082F77
:10A380007FD126E00027EEE70227ECE70427EAE783
:10A39000FDF77AF806E00968C90605D4304603E0FF
:10A3A000FDF792F8002872D062685100511881427E
:10A3B00067D81103814264D3010E060250080023BE
:10A3C00030185941FAF7AAFE03210902411A384A06
:10A3D00055E00120C003E7E70122E369D20393427D
:10A3E0002BD13B0000F0E1F90906090C4D114D4D50
:10A3F0004D274D00FDF748F809E0FDF755F806E058
:10A400000968C90605D4304603E0FDF75DF8002869
:10A410003DD0616840004A088018FAF769FE80B2B2
:10A420000146244A103991422BD8511C01400007A3
:10A43000400F084329E01046EBE73B0000F0B5F978
:10A440000906090C2112212121232100FDF71CF806
:10A450000AE0FDF729F807E00968C90606D4304686
:10A4600004E00EE0FDF730F8002810D061684A08DB
:10A470001018FAF73DFE80B201460E4A103991429B
:10A4800003D9012503E01046F0E72168C8600020E9
:10A490006066A0662846F8BD00480040F369FFEFFB
:10A4A00000380140401002400044004000093D00D7
:10A4B000FFFC0F00EFFF0000F8B504464165403097
:10A4C00000262746028380373E602220E06725462B
:10A4D000206F603500281CD01749C162216F1748D2
:10A4E0000863216F16484863206F8663236F606D91
:10A4F0009C4613462168024660462431FCF7B6F9B3
:10A50000002806D0102038602E752020A06701207A
:10A51000F8BD2E7520680168FF22013211430160E9
:10A52000206881680122114381602068816840228F
:10A53000114381600020F8BD99A10008F7A100082F
:10A540004DA10008FFB581B005460F4604466035B1
:10A550000A9E39E0701C37D0FCF730FB0499401A92
:10A56000B04222D8002E20D02068016849072BD5A0
:10A57000C069C043000527D401202168C0020862D9
:10A5800020680168FF22A132914301602068816840
:10A590004908490081602020A067E067803420607E
:10A5A00000202875032005B0F0BD20680168FF2257
:10A5B000A1329143016020688168490849008160A7
:10A5C0002020A067E067EBE72068C1693846884330
:10A5D00005D0002103988142BCD00020E3E701218F
:10A5E000F8E7000010B50449102009680862024825
:10A5F000FDF72AFC10BD0000CC16002001490D20FB
:10A60000887070475400002010B5FEF7A1F9FEF7DE
:10A61000B9FAC82202490348FDF7C6FD10BD000083
:10A62000200D0020CC160020F8B53E4C00232178E8
:10A630003D4A1D46082910D0072947D0062950D089
:10A64000052952D0042953D0032954D0002956D0CB
:10A65000012958D002295AD05BE0A17800264A1F70
:10A6600004E0314FBF5DFB189BB2761C9642F8DBCD
:10A67000667927799A195118E3786278C918891888
:10A68000C9194018C0430006000E1AD1012E14D07B
:10A69000022E16D125482449C018FAF76FFD01F0A3
:10A6A00087FF642000F0A6FABFF34F8F21492048AE
:10A6B000C860BFF34F8F00BFFDE759081046FFF792
:10A6C000B7F92570E570A570A571F8BDA179505452
:10A6D000491CC8B2A071A178491F8842F5D1082051
:10A6E00001E0607007202070F8BDE0700620FAE7F6
:10A6F00060710520F7E7A070E5700420F3E75528A6
:10A7000007D10120EFE7AA2803D10220EBE70328B5
:10A7100003D02570E570A570F8BD0320207020716E
:10A72000F8BD000034010020DE140020E80D0020F8
:10A730000400FA0500ED00E010B5024A024900F0FD
:10A74000E5F910BDF5B80008880100202021020CB1
:10A7500001D010211046020A01D010460839020922
:10A7600001D01046091F820801D01046891E4208F8
:10A7700001D0881E7047081A7047F8B5040C8BB2D8
:10A78000264682B25E430D0C1046370C5843360401
:10A7900080190021794116466E43370C3604801922
:10A7A000794126466E438919F8BD30B47446641E5B
:10A7B0002578641CAB4200D21D46635D5B00E31844
:10A7C00030BC18474900CA020243100000D00420E0
:10A7D0004A0D01D001221043044A490D914201D192
:10A7E00002210843012800D105207047FF0700001F
:10A7F0008307FF22DB0E9A408907090E9940002843
:10A8000008DB830809489B001B181868904308431D
:10A81000186070470007000F0838830804489B0041
:10A820001B18D86990430843D861704700E400E0E2
:10A8300000ED00E0BFF34F8F04490348C860BFF349
:10A840004F8F00BFFDE700000400FA0500ED00E0B7
:10A85000F8B504464F1EC8000838211815461E4694
:10A86000086849683A4606239A4310D02A46334678
:10A87000FAF70AFE3A46D200083AA3181A687F1E71
:10A880005B68FAF74FFD06223B469343EED1022F59
:10A8900023D0042F11D0062F2FD12A463346FAF7A2
:10A8A000F3FDE36AA26AFAF73DFD2A463346FAF75A
:10A8B000EBFD636A226AFAF735FD2A463346FAF75A
:10A8C000E3FDE369A269FAF72DFD2A463346FAF75C
:10A8D000DBFD63692269FAF725FD2A463346FAF75C
:10A8E000D3FDE368A268FAF71DFD2A463346FAF75E
:10A8F000CBFD63682268FAF715FDF8BD002210B59C
:10A90000134610460149FAF727FE10BD0000F03F3C
:10A9100010B5FAF707FD10BD002210B5134610461A
:10A920001146FAF719FE10BD10B50721024A0020A2
:10A930000907FAF789FE10BD01030000034A10B5AC
:10A9400000201107FAF780FE10BD000001FDFFFF97
:10A9500002E008C8121F08C1002AFAD170477047E8
:10A96000002001E001C1121F002AFBD17047000046
:10A9700001490860704700008C01002008B50021E3
:10A98000684601706B46012202212C2000F052FF24
:10A990000221684601706B4601222C2000F04AFF1C
:10A9A00008BD000038B504466D20694608706B4646
:10A9B000012207492E2000F03DFF0649002C01D05E
:10A9C000054A00E0054A2E2000F01AFF38BD0000BD
:10A9D0000608000006180000070600000716000021
:10A9E00038B504466B4602220021362000F0EEFD09
:10A9F000B3212300FFF7D9FE0E0F08153A3A3A3A71
:10AA00001C273A3A2F34483A0021684601704078B2
:10AA10004108490014E06946087880088000401C1D
:10AA200004E06946087880088000801C08701DE0FA
:10AA3000684602780A40483202704178802001431B
:10AA40006846417012E0684602780A400270407819
:10AA50004106490EF4E7694648780221084303E0BD
:10AA600069464878FD210840694648706B460122D6
:10AA70000021362000F0DEFE012200AB1146362018
:10AA8000013300F0D7FE38BD69460878CF21084071
:10AA900069462030CAE708B50321684641700121A4
:10AAA00001706B4602220021362000F0C3FE012215
:10AAB000D20306212D2000F0A3FE012000F09AF819
:10AAC0000120FFF78DFF08BD08B5020A69464A70EC
:10AAD00008706B46022204212D2000F0ABFE0320FB
:10AAE000694608706B46012206212D2000F0A2FE67
:10AAF0000020694608706B46012206212D2000F0D7
:10AB000099FE0A212D2000F047FD08BDF8B5164634
:10AB10000F460446002503E03946B047641C6D1C0F
:10AB200020780028F8D12846F8BD0000F8B54A0082
:10AB30002B4B520DD6182B4A0C460546142E2BDAF9
:10AB4000002E12DA284BFAF7EDFB00221346FAF733
:10AB500043FE40D2002C03DA0124E40700253AE04A
:10AB60002046284337D0214C14E0214F0B46F740B4
:10AB70003B402B4331D01C4BFAF7D4FB0022134649
:10AB8000FAF72AFE27D2002C03DD01200005F04051
:10AB90000419BC4300251EE0332E1EDC334600277B
:10ABA000143BFF43DF40384217D00F4BFAF764FCE9
:10ABB00000221346FAF710FE0DD2002C0ADD142EE7
:10ABC0000CD03420811B012088404019A84200D2BB
:10ABD000641C0546BD4321462846F8BD641CF9E7C0
:10ABE00001FCFFFF9C7500883CE4377E0000F03FCD
:10ABF000FFFF0F007D2110B5C900484300F001F8A8
:10AC000010BD002140E000BF00BF00BF00BF00BF7B
:10AC100000BF00BF00BF00BF00BF00BF00BF00BF3C
:10AC200000BF00BF00BF00BF00BF00BF00BF00BF2C
:10AC300000BF00BF00BF00BF00BF00BF00BF00BF1C
:10AC400000BF00BF00BF00BF00BF00BF00BF00BF0C
:10AC500000BF00BF00BF00BF00BF00BF00BF00BFFC
:10AC600000BF00BF00BF00BF00BF00BF00BF00BFEC
:10AC700000BF00BF00BF00BF00BF00BF00BF00BFDC
:10AC800000BF00BF00BF491C8142BCD37047FFB565
:10AC900081B01E460F46040026D00B99039801434D
:10ACA000A06A3943826807209047002818DB0A9978
:10ACB000A06A3143826806209047002810DB2546B1
:10ACC0002035A979032F01D908200143032E01D98A
:10ACD00004200143A06A826809209047002806DA10
:10ACE0000120C04305B0F0BD0020C043FAE738465C
:10ACF00000F000F92060304600F0FCF860600A982F
:10AD000068700398A870EF702E710B98687100201E
:10AD1000E8E70000F7B50446002090B000900190ED
:10AD2000002C05D06A46062101F07CFC062803DAD7
:10AD30000020C04313B0F0BD684640780102684669
:10AD4000007800040918684680780818FAF7B8FCFB
:10AD5000054668460391007901026846C078000400
:10AD60000918684640790818FAF7AAFC0322064633
:10AD70000F4692075C4BFAF72FFD07D200225B4B80
:10AD800030463946FAF772FB06460F460322920711
:10AD9000554B28460399FAF71FFD07D20022534B63
:10ADA00028460399FAF762FB054603912068FAF7F3
:10ADB00087FC02460B4630463946FAF7CDFB07467C
:10ADC0000A200791205EFAF767FC3A46079BFAF7DC
:10ADD0005BFB064608200991205EFAF74BFC002138
:10ADE000C943FAF793FAFAF7CFFC3246099BFAF710
:10ADF00099FA069108906068FAF762FC02460B46E1
:10AE000028460399FAF7A8FB05461A200E46205E4D
:10AE1000FAF742FC2A463346FAF736FB0C900991C2
:10AE20001620205EFAF738FC099B0C9AFAF77AFA9A
:10AE300005910A902A46334638460799FAF724FBCB
:10AE4000059B0A9AFAF720FB05910A901420205ED0
:10AE5000FAF722FC3A46079BFAF716FB07461C2036
:10AE60000791205EFAF718FC2A463346FAF70CFBE6
:10AE70000E900B911820205EFAF70EFC0B9B0E9A99
:10AE8000FAF750FA2A463346FAF7FEFA0B910E907B
:10AE90002069FAF701FC0B9B0E9AFAF743FA2A464F
:10AEA0003346FAF7F1FA05460E46E068FAF7F4FB86
:10AEB0002A463346FAF736FA3A46079BFAF732FA49
:10AEC000059B0A9AFAF72EFA01229207084BFAF725
:10AED000DBFA02460B46129C0898069903C41198A7
:10AEE0000CC0002026E70000FFFF5F41000070411A
:10AEF000E17A843F00B50121C9040300FFF755FC46
:10AF0000081A05080B0E1114171A0320C00400BDFF
:10AF10000720C00400BD0F20C00400BD1F20400357
:10AF200000BD3F20400300BD7F20400300BDFF2047
:10AF3000400300BD084600BDFEB5264F0D46040087
:10AF40000FD0002D0DD0264600202036B071F071B4
:10AF500029680D208847002801DA7800FEBD1028F6
:10AF600001D03846FEBDA562E968002901D028203D
:10AF70008847204600F030F80028F3DBA06AA521BE
:10AF800082680E209047A06A962182680F20904721
:10AF9000A06A0221826862209047A06A002182682C
:10AFA0000E209047A06A002182680F209047717997
:10AFB0003020019100900623202201212046FFF736
:10AFC00066FE0028CEDB204600F0AEF80028C9DB84
:10AFD0000020FEBDFFFFFFFF10B586B00446142120
:10AFE0006846FAF7E4F8002C7ED0A06A1221436884
:10AFF0006A4610209847122877D1684600780122C7
:10B00000010168464078120300090818434920816D
:10B01000884201DD801A20816846837840780007E5
:10B02000000D18186081884201DD801A6081684631
:10B030000079012201016846C07812050003091851
:10B0400068464079000908183549E060884201DD0A
:10B05000801AE060684640790007030B68468079F3
:10B0600000021B186846C07918182061884201DD6B
:10B07000801A20616846417A007A0002081802B2FC
:10B08000284801210904A282824201DD521AA282CB
:10B090006A46D37A927A12029A1812B2E2828242F5
:10B0A00001DD521AE2826A46537B127B12029A1821
:10B0B00012B22283824201DD521A22836A46D37B76
:10B0C000927B12029A1812B26283824201DD521AF6
:10B0D00062836A46537C127C12029A1812B2A283CF
:10B0E000824204DD501A01E00BE008E0A083A06A70
:10B0F000016828208847002806DA0120C04306B0EE
:10B1000010BD0020C043FAE7C011C007203400285A
:10B1100000D0802060710020F1E70000FF070000F0
:10B12000FFFF0700FF7F000010B5040009D0A06AF0
:10B130000721826808209047002805DA0120C043D3
:10B1400010BD0020C04310BD072020342070002017
:10B1500010BD0000FEB5044600200190009060790B
:10B16000734940000E5A61782578491E7148CFB264
:10B170000163042D77D0072D75D00021029121782D
:10B1800001736C49E379012292058969002B6CD027
:10B19000914381616748217A4173217A82698907E5
:10B1A000890B0A4382610021042000F034FB3246FF
:10B1B00061492E2000F024FB3846FFF7F3FB5F4E79
:10B1C0000522705D810040185D49431807212B203E
:10B1D00000F030FB5B49029801220B180B2128205C
:10B1E00000F028FB705D584980000A580C21282087
:10B1F00000F011FBE079554980004018A179490021
:10B20000425A0221272000F0FBFA51487E00825B5F
:10B210000421272000F0F4FAE079002829D0A07852
:10B2200004282CD0282069460872202206212720D5
:10B2300000F0E6FA02AB01222621272000F0FAFAFC
:10B24000444938014018E1788900425808212720F4
:10B2500000F0E1FAA17A601C627A0902114313D06E
:10B2600016E000E001E0012188E71143F608816162
:10B2700090E764220621272000F0C2FAE0E71020C0
:10B28000694608720246D1E733490172090A4172E0
:10B29000417A007A0A0202432021272000F0B0FA06
:10B2A0002E4F0C2123203A6800F0B5FAF01982885D
:10B2B0000421232000F0A4FAA07900280BD0E07923
:10B2C0002749012243180021212000F0B3FA03206E
:10B2D0000190012000902A07120F100102436078AC
:10B2E00000218007000B02430198000502430098EB
:10B2F000400402432079C006400902436079C00639
:10B3000002431F2000F087FAA078617801230843E8
:10B3100002040848DB030261E179490319430A4347
:10B3200002610021082000F076FA0020FEBD000036
:10B3300058C70008BC0100200428000000C700080E
:10B34000240000204200002008C7000828C7000889
:10B3500034C7000838C700084110000020C70008A3
:10B360004400002038B50C4607498A8B002102436F
:10B370002C2000F045FA684604706B460122062135
:10B380002C2000F057FA38BDBC01002010B5FFF7A3
:10B39000F5FA10BD10B504460421362000F0FCF883
:10B3A0000121C902002C01D0084300E08843024675
:10B3B0000421362000F02FFA10BD000038B54020DF
:10B3C0006946087000210E2000F0E6F804460022CD
:10B3D00011460E2000F01FFA6B46012200210D20BD
:10B3E00000F028FA074A00210F2000F014FA00F0BC
:10B3F000EDF9224600210E2000F00DFA024800214E
:10B40000017338BDF8FF2724DC010020FEB5054696
:10B41000042069460870514C002060752146203197
:10B42000206348710873A0836063A06300F0C8F8CC
:10B430004B4E206002E000F0C3F82060B042FAD129
:10B440000020FFF7CDFA00F0BBF8464E20603078C0
:10B45000242801D9243806E00621F9F749FE0622FE
:10B46000101A40010843020601040A4301020A437C
:10B470000243B260706000211E2000F0CCF900F0A1
:10B480009FF820606B4601220021242000F0D2F9B1
:10B490001E20FFF719FB86B2300AA0730420FFF7C5
:10B4A00013FB074600F08CF820603806000E0DD024
:10B4B00002206946087101AB012212212D2000F003
:10B4C000B9F9A08B012109030843A08300F078F8A3
:10B4D00020600620FFF7F8FA60600720FFF7F4FA13
:10B4E000A060F006C00E207501D110202075C0B2FA
:10B4F00000F0DCF9E80707D0FFF7CDFAA08B0121B7
:10B50000C9020843A0830AE00521362000F02EF886
:10B510001549084002460521362000F071F9012046
:10B52000FFF75EFA0021042000F036F8A061002148
:10B53000262000F031F81521890308430246002136
:10B54000262000F068F900222621362000F058F964
:10B5500000F036F820600020FEBD0000BC01002095
:10B560003001CADE18000020FFFD000038B5094C8C
:10B5700089B280B26B46022200F028F8002806D17A
:10B5800068464078010268460078081884B2204670
:10B5900038BD0000FFFF000038B50024E44389B245
:10B5A00080B26B46042200F011F8002806D1032176
:10B5B0006846435C2202D418491EFAD5204638BD9D
:10B5C00010B500210846FFF7E7FF10BD38B5002988
:10B5D00009D0402420436C462070C8B27F2906D889
:10B5E000607002200AE069460870012006E08024AD
:10B5F00020436C466070C809A0700320694600F0C3
:10B60000B1FF38BD10B5144603460A462146112045
:10B61000FFF7DCFF10BD10B5034605220021152001
:10B62000FFF7D4FF10BD10B50346052200211720F7
:10B63000FFF7CCFF10BD38B50546002069460870FD
:10B6400000F0C4F8FF2401342246002D01D003226B
:10B65000120200210D2000F0D3F8002D13D06B460C
:10B66000012203210F20FFF7B1FF68460078000791
:10B6700009D5FFF7A3FE224600210D2000F0C0F8F7
:10B680000020C04338BD002038BD10B5024601215E
:10B690000A2000F0C0F810BD10B5044600211A20A1
:10B6A000FFF77AFF000D22030005120B0243002171
:10B6B0001A2000F0B0F810BD10B5024602492E2045
:10B6C00000F09EF810BD000004180000F8B5054613
:10B6D0006B46012203210420FFF778FF0126114C5D
:10B6E0003607002D0DD02A4600210C2000F088F8E6
:10B6F000694608781021084369460870A0693043FC
:10B7000007E069460878EF21084069460870A0699B
:10B71000B0430B46A06101220321042000F08AF807
:10B72000F8BD0000BC01002010B502460021182021
:10B7300000F066F810BD0000F8B507460025684621
:10B740000570B807204C2E4600280ADA802069468A
:10B7500008706B46012200210D2000F06BF80120DB
:10B760002073F8076946087821D006210843694606
:10B7700008706B46012200210D2000F05BF80321C8
:10B780000F20FFF7F3FE8121C900084219D04020A5
:10B79000694608706B46012200210D2000F04AF82E
:10B7A0000020FFF7F7FD00252673ED4309E0022195
:10B7B0000843694608706B46012200210D2000F005
:10B7C00039F82846F8BD0000DC0100201CB56B46A6
:10B7D000012203210F20FFF7F9FE6846007840227E
:10B7E000C1091040C9014000814208D001206946CA
:10B7F0000871024601AB03210D2000F01BF81CBDAF
:10B8000008B56B461A70120A5A7089B280B20222C9
:10B8100000F010F808BD38B500236C46E254120A57
:10B820005B1C042BFADB89B280B22346042200F0B1
:10B8300001F838BD38B58024002909D0C025284337
:10B840006D462870C8B27F2907D86870022009E0C9
:10B85000204369460870012004E020436870C8094D
:10B86000A8700320694600F027FF38BD10B51446C4
:10B87000012312189B029A4202D90020C04310BD36
:10B880000B46821E21460920FFF7D4FF002010BD81
:10B8900010B5054A8905126901430A4300210820B1
:10B8A000FFF7B9FF002010BDBC01002038B50446E9
:10B8B0006B4601220E212B20FFF788FE6846007898
:10B8C000E10640094001C90E0143684601706B461C
:10B8D00001220E212B20FFF7ADFF38BD10B500214E
:10B8E00042541C06120A22431B0A491C0429F7DB96
:10B8F00010BD000013B501231A4669460248FCF743
:10B9000085FC00981CBD0000CC1600207CB50024EE
:10B9100025466846FFF77FFE04206946220E2D0269
:10B92000154322020C5C1443401EF7D520462946DD
:10B930007CBD7CB5002425466846FFF774FE0420D4
:10B940006946220E2D02154322020C5C1443401E50
:10B95000F7D5204629467CBDFBF73EF9FEF708F9EE
:10B96000FDF70AF83E493F48002522C00560856181
:10B97000C5613D490562C1600838FBF7BFFAFCF7B5
:10B98000E7FFFDF7FFF8FDF79BF8FCF7ADFF052497
:10B9900001222407D1032046FBF709F9FDF798FEA1
:10B9A000FCF79AFEFAF7FAF8FAF77CF9FAF74AF98F
:10B9B000FCF7AEFC0721A015FFF7D4FCFFF7E6FC6F
:10B9C000012211032046FBF7F2F82648C822274936
:10B9D000C830FCF7E9FB264F264E274C3878002864
:10B9E0000FD13078002801D003280AD10121C902E3
:10B9F0002248FBF7CFF8002803D101210846FBF7C6
:10BA000091FBE078002828D06078002825D0E570E8
:10BA100072B620780F280AD90120184900038861DE
:10BA2000FEF7F4F901201549000388620CE00122B9
:10BA300051031248FBF7BBF8FEF7E8F90121002299
:10BA400049030E48FBF7B3F862B6FCF76BFD208C98
:10BA50000028C3D0401E2084C0E7FCF763FDBDE78B
:10BA6000007C004004160020FFFF0000200D002095
:10BA70005A000020810000203C01002000040050FA
:10BA800010B586B01748FBF7BCF914216846F9F7E2
:10BA90008EFB1548009003200190002002900520A5
:10BAA00069460007FAF7BAFF69461048FAF7B6FF89
:10BAB00069460F48FAF7B2FF01210846FBF732FB4F
:10BAC000FF2401342046FBF705FB0A4908680422DD
:10BAD000104308602046FBF70DFBFBF713FB06B095
:10BAE00010BD000004160020FFFF000000040050FD
:10BAF000000800500070004010B501229202174962
:10BB00001748FAF753F91548164902888A4223D094
:10BB1000018004218180FF21F531C1800A2101814A
:10BB200000211E224181D24382810122C281818370
:10BB30004323C38602230387782343878287C287F0
:10BB400002464032118451849184C1839180142330
:10BB50008382118200F02CFD10BD0000E80D002052
:10BB600000FC0008AA550000F0B51FB496B084464A
:10BB70000C460246199D189803904900680063001E
:10BB8000490840080193002A01D0012600E0002660
:10BB90009E19FE4BF6185B109E422BD36E00039F3E
:10BBA0000296002F00D00127F719F84EF84BBE1966
:10BBB0009E421FD3039E0346F64F334309D03B46B4
:10BBC0009C4201D1002A04D0019B002A05D0012605
:10BBD00004E0002039461BB0F0BD00269E19EE4B54
:10BBE0009E4207D8039F029E002F00D00127F6191E
:10BBF0009E4207D92B4660462146189AFEF788FEDA
:10BC00001BB0F0BD0023002C29DAE44EB04226DA46
:10BC1000E34EB04201DB022321E0DE4EB0421EDBE8
:10BC2000E04E070DBE19142E09DD3427BF1B039EFD
:10BC3000FE400196BE40039FBE420BD00FE0039F23
:10BC4000002F0CD11427BF1B0646FE400196BE40B4
:10BC5000864204D1019BDE07F60F02239B1B0E4692
:10BC6000164318D1002D16DA002C03D0022B01D078
:10BC7000012B06D00220FEF77BFEFEF73FFE1BB035
:10BC8000F0BD0220FEF774FEFEF738FE0122D20757
:10BC900051401BB0F0BD039E002E61D1BF4EB0429B
:10BCA00020D1C148844201D1002A08D0B94881423C
:10BCB00009DB002D10DB189829461BB0F0BD0020D1
:10BCC000B4491BB0F0BD002D06DA01222946D20787
:10BCD000189851401BB0F0BDB449794408684968D0
:10BCE0001BB0F0BDAB4FB84225D1002D1FDA0029A3
:10BCF00004D0B14212D1002A09D018E0002A72D132
:10BD0000A649E20F0020D20711431BB0F0BD00206E
:10BD1000E20F0146D20711431BB0F0BDB14206DA73
:10BD2000234600203946F9F717FC1BB0F0BD10463A
:10BD300021461BB0F0BDB14212DA0126B607B5426A
:10BD400003D1234610461946FEE3994EB54207D16A
:10BD5000261E05DB1046314600F040FC1BB0F0BD4E
:10BD600067007F081646002A40D100290AD08B4A76
:10BD7000914229D1002C0EDD002D1CDB0020114644
:10BD80001BB0F0BD022B16D0002C14D0012B12D109
:10BD9000002C14DB0FE0002C28DA002D09DB012B2E
:10BDA00003D000207D491BB0F0BD002081491BB0AD
:10BDB000F0BD012B03D0002001461BB0F0BD0020D8
:10BDC0000121C9071BB0F0BD724A91420ED1002C6F
:10BDD00001DA002B17D0022B06D00020C043F9F760
:10BDE0005BFC1BB0F0BD90E20120F8E7E217521CAB
:10BDF00094461A4307D000220892664C62465B1EA6
:10BE00001A4307D009E00120FEF7B2FDFEF784FDDA
:10BE10001BB0F0BD0022644C0892674A90427DDD61
:10BE2000664B674A98421FDD914202DC002D05DB1C
:10BE30004DE05848814217DB002D48DD0220FEF717
:10BE400097FDFEF771FD05460E460022534B214635
:10BE50000898F9F719FB084671004908C00FC00798
:10BE6000014328461BB0F0BD914215DA002D2EDAB1
:10BE70000220FEF77DFDFEF757FD05460E46002227
:10BE8000464B21460898F9F7FFFA72005208C80F8E
:10BE9000C0070243114617E03E4B994223DD002DB7
:10BEA00015DD0220FEF764FDFEF73EFD05460E4659
:10BEB00000223A4B21460898F9F7E6FA0846710045
:10BEC0004908C00FC007014328461BB0F0BD02203F
:10BED000FEF74EFDFEF732FD49004908E20FD2079A
:10BEE00011431BB0F0BD002230463946F9F7BEFAC7
:10BEF000012205460E46D243F9F7A6FB314A324BE2
:10BF0000F9F7BAFA2A463346F9F7BEFA0022284B67
:10BF1000F9F7B2FA07462A46334600E064E0039197
:10BF200010461946F9F7B0FA3A46039BF9F7ACFA0E
:10BF30000746032209915207244B28463146F9F758
:10BF4000A3FA07910C90224A204B38460999F9F739
:10BF50009BFA074601911F4A1F4B28463146F9F7C5
:10BF600093FA3A46019BF9F781FA07460B460246D7
:10BF7000099107990C98F9F7D5F900250E4628463E
:10BF8000079B0C9AF9F772FA3A4627E0FFFF1F0069
:10BF9000FFFF0F000000F03F0000E0FF0000F07F17
:10BFA0000000404301FCFFFF0000F0BF5A0B0000FF
:10BFB0000000E03F0000F0FF0000E0410000F0431F
:10BFC000FFFFEF3F555555555555D53F4715F73FA1
:10BFD000FE822B6544DF5DF80BAE543E099BF9F7FA
:10BFE0004BFA02460B4652E1012500202D05A942DD
:10BFF00007DA352230463946F9F726FB0646342063
:10C00000C0430A151218FE48101803900803FD4992
:10C01000000B01430F46FC49884201DC002003E08D
:10C02000FA49884202DA0120119005E000201190BF
:10C030000398401C7F1B039011980597C200F44899
:10C040000F927844801843680268394630460D9351
:10C050000292F9F70BFA07910C9030460D9B029A69
:10C060000599F9F75FF902460B460020E549F9F713
:10C0700073FA09910490079B0C9AF9F705FA12904C
:10C0800000201090E3480D46784400680E9001218E
:10C0900078104907084311990D9B89044018012124
:10C0A000C90447183946029A0E98F9F7DFF9324663
:10C0B000059BF9F7E1F902460B4629461098F9F776
:10C0C000E3F9064602913B4629460E9A1098F9F785
:10C0D000DBF9079B0C9AF9F7CFF93246029BF9F787
:10C0E000C5F9099B049AF9F7CFF90591129A0A90BC
:10C0F0002B4610461946F9F7C7F906460246C648C8
:10C100000F460B4606217844FEF7A2FB32463B461B
:10C110000091049010461946F9F7B6F9009B049A6D
:10C12000F9F7B2F906460F462B461946129A1098AF
:10C13000F9F7F8F8059B0A9AF9F7A6F932463B4653
:10C14000F9F7F0F8109A079104902B46104619461B
:10C15000F9F79AF9B14E0022334609910290F9F7A6
:10C16000E1F8079B049AF9F7DDF80020074602463C
:10C1700033460091F9F77AF9099B029AF9F776F9B3
:10C18000079B049AF9F778F906460D913A46294635
:10C19000009B1098F9F778F907910C902B463046E0
:10C1A000129A0D99F9F770F905460E463A46009B2A
:10C1B00005990A98F9F768F933462A46F9F7B2F86B
:10C1C00002460B460746099107990C98F9F7AAF819
:10C1D00000250E462846079B0C9AF9F747F93A4680
:10C1E000099BF9F749F907460722099152078C4B39
:10C1F00031462846F9F748F907910090894A884B5B
:10C2000038460999F9F740F907460191864A874B64
:10C2100031462846F9F738F93A46019BF9F782F892
:10C22000834B7B440F9A9B181A685B68F9F77AF87E
:10C23000029009910398F9F72FFA05910490099B50
:10C24000029A07990098F9F76DF87A4B7B440F9A98
:10C250009B181A685B6817460393F9F763F8059B08
:10C26000049AF9F75FF80E462846059B049AF9F7F9
:10C27000FDF83A46039BF9F7F9F8079B009AF9F79E
:10C28000F5F8099B029AF9F7F7F802460B46199957
:10C2900000200C900F461898F9F7F6F802910490D8
:10C2A0003B460C9A19991898F9F7E0F82A46334654
:10C2B000F9F7EAF8029B049AF9F734F809910E901D
:10C2C0002A46334639460C98F9F7DEF806460F46FB
:10C2D000099B0E9AF9F726F8574A0D46914220DB42
:10C2E0005242AA18024310D132463B46F9F7BEF833
:10C2F00004900391514A524B09990E98F9F712F89C
:10C30000039B049AF9F768FA1ED20220FEF730FB6D
:10C31000FEF70AFB49004908E20FD20711431BB0A0
:10C32000F0BD6A00474B52089A420DD3464AAA18FC
:10C33000024300D0CBE532463B46F9F797F8099B1C
:10C340000E9AF9F749FAF5D96800002340082C49FC
:10C350000393020D3D4B5218984223DD0120000546
:10C36000521CD04042195000400D401838497944C1
:10C37000096813468C463749C1408B43120301219B
:10C38000120B090551181422101AC1400391002DF7
:10C3900001DA48420390624630463946F9F766F8BA
:10C3A00006460F4632463B4609990E98F8F7BAFF03
:10C3B00000252A46284B28460591F9F765F807918C
:10C3C0000C90264A264B28460599F9F75DF800910E
:10C3D000029032463B4628460599F9F747F8099BF3
:10C3E0000E9AF9F749F81F4A1F4BF9F74DF8009BD1
:10C3F000029AF8F797FF07460B460246099135E087
:10C4000001FCFFFF0000F03F8E9803007AB60B009E
:10C410006A070000AC070000D606000000000840D4
:10C4200009C7EE3FFD033ADCF5015B14E02F3EBE89
:10C43000AA0500007005000000009040FE822B65F8
:10C440004715973C00CC904000346F3F0000E03F20
:10C45000C6040000FFFF0F00432EE63F396CA80C16
:10C46000615C20BEEF39FAFE422EE63F07990C9838
:10C47000F8F758FF05460E46079B0C9AF8F7F6FFAB
:10C480003A46099BF8F7F8FF09912A4633460E9081
:10C4900010461946F8F7F8FF074602462F480B46A4
:10C4A000059105217844FEF7D3F93A46059BF8F744
:10C4B000EBFF2A463346F8F7DFFF0746019128468F
:10C4C0003146099B0E9AF8F7DFFF099B0E9AF8F7A1
:10C4D00029FF012304910C9000229B073846019903
:10C4E000F8F7C4FF05910E903A4628463146019B65
:10C4F000F8F7CAFF059B0E9AF9F72EF8049B0C9AE1
:10C50000F8F7B4FF2A463346F8F7B0FF0022144B81
:10C51000F8F7B2FF064603980D46000541190915C4
:10C52000002912DC30462946039AF9F78DF8FEF708
:10C5300049F9042801D1FEF701FA30462946039A49
:10C54000F9F782F8064601E004E029180B46324666
:10C5500021460898F8F798FF1BB0F0BD680300006B
:10C560000000F03FF0B58C46002510260521090794
:10C570008E620E4C08E067467F5DE760A768FF07A4
:10C58000FCD0E7681F706D1C8542F4DB0020074675
:10C5900006E0E760A568ED07FCD0E5681D54401C87
:10C5A0009042F6D38E610020F0BD000000300140C3
:10C5B00070B572B60124074DA40221462846F9F74A
:10C5C000DBFB002804D0224603492846F9F778FC13
:10C5D00062B670BD00FC0008E80D0020F8B5064604
:10C5E0000C46F9F707FA051E0F4600D0012001435B
:10C5F00049000B484908411AC90F0DD0002E01D03F
:10C60000012100E000210C4361004908401AC00FDD
:10C6100002D10120FEF7ACF928463946F8BD0000EA
:10C620000000F07FF8B515460E460746002407E0E7
:10C630003819C0B200F008F8641C2870E4B26D1C10
:10C64000B442F5D33046F8BD10B50446FBF706FFFB
:10C65000EE20FBF7D6FEFBF73AFF2046FBF7D1FEB4
:10C66000FBF735FFFBF7FAFEEF20FBF7CAFEFBF7FF
:10C670002EFF0020FBF798FE0446FBF70AFF20463A
:10C6800010BD704770B50D460446FBF7E7FEEE207F
:10C69000FBF7B7FEFBF71BFF2046FBF7B2FEFBF7ED
:10C6A00016FF2846FBF7ADFEFBF711FFFBF7F1FE87
:10C6B0000A20FEF7A6FA70BDF0B500251026052762
:10C6C0009C463F070B46BE620C4C06E0595DE1609C
:10C6D000A168C907FCD0E1686D1C8542F6DB00202B
:10C6E00007E06146095CE160A168C907FCD0E16828
:10C6F000401C9042F5D3BE610020F0BD00300140E7
:10C700000000010203040005405C0000A05C04007E
:10C71000C06C0800805C0400E03F1E00E07D1E004D
:10C7200007A9022570889B880A00160001000600F0
:10C730000100020087008D002D001A3152001A33CB
:10C740009A001A351D011A376B003B31BE003B338E
:10C750005E013B3596023B37000099599959EB51E0
:10C760008F421E45142E0080EB51F5283333E13AF9
:10C77000703DE13AC235852BC2353333C235C235FF
:10C78000AE47E13A5138A3305138000000000000B4
:10C7900000000102030406070809030406080C1040
:10C7A0001820300000000001020304000000000017
:10C7B000000000000000F03F000000000000F83F13
:10C7C00000000000000000000000004003B8E23F4D
:10C7D000000000000000000006D0CF43EBFD4C3EFF
:10C7E000033333333333E33FFFAB6FDBB66DDB3FF4
:10C7F0004D268F515555D53F01411DA96074D13F3C
:10C8000065DBC9934A86CD3FEF4E454A287ECA3F35
:10C810003E5555555555C53F93BDBE166CC166BFB7
:10C820002CDE25AF6A56113FF16BD2C541BDBBBEB0
:10C83000D0A4BE726937663E000000000000000010
:10C8400060C800080000002090010000BC5A0008E9
:10C85000C4C8000890010020681A000060A9000800
:10C860000124130704380D091E0805400826091085
:10C870004008560A131D043B08BE0516D8BC4010DC
:10C880000852010338C842077252030CE5800C1BA2
:10C890000202DD140901022281F01F6681049889D9
:10C8A0009686967982159803981498879674977847
:10C8B00082439788967197778249F10139293F928F
:04C8C00004922000BE
:04000005080050C1DE
:00000001FF
